:020000040000FA
:100000000C9455010C947D010C947D010C945F259A
:100010000C945F250C945F250C947D010C947D015C
:100020000C947D010C947D010C947D010C947D0158
:100030000C947D010C947D010C947D010C947D0148
:100040000C9415250C947D010C94E3240C94BD2490
:100050000C947D010C947D010C947D010C947D0128
:100060000C94D7250C947D0107634236B79BD8A723
:100070001A39685618AEBAAB558C1D3CB7CC5763CD
:10008000BD6DEDFD753EF6177231BF000000803F7B
:1000900008000000BE922449123EABAAAA2ABECD97
:1000A000CCCC4C3E00000080BEABAAAAAA3E000009
:1000B0000000BF000000803F000000000008417801
:1000C000D3BB4387D1133D190E3CC3BD4282AD2B38
:1000D0003E68EC8276BED98FE1A93E4C80EFFFBE30
:1000E00001C4FF7F3F00000000004E414E494E49D1
:1000F0005459494E46CDCCCC3D0AD7233C17B7D1F5
:100100003877CC2B329595E6241FB14F0A0000209A
:10011000410000C84200401C4620BCBE4CCA1B0E19
:100120005AAEC59D7400407A10F35A00A0724E1862
:10013000090010A5D4E80000E87648170000E40B99
:1001400054020000CA9A3B000000E1F5050000805F
:10015000969800000040420F000000A086010000B9
:1001600000102700000000E8030000000064000009
:100170000000000A00000000000100000000002C48
:1001800076D888DC674F0823DFC1DFAE59E1B1B70D
:1001900096E5E3E453C63AE651997696E8E6C284DA
:1001A00026EB898C9B62ED407C6FFCEFBC9C9F40F2
:1001B000F2BAA56FA5F490055A2AF75C936B6CF917
:1001C000676DC11BFCE0E40D47FEF520E6B500D0ED
:1001D000ED902E0300943577050080841E08000002
:1001E000204E0A000000C80C333333330F986E12D0
:1001F000831141EF8D2114893BE65516CFFEE6DBD6
:1002000018D1844B381BF77C1D901DA4BBE424201F
:100210003284725E228100C9F124ECA1E53D274CB5
:100220004F470056455200005EBCE2613FDD83C28D
:100230009C7E20A3FD1F41009D23BE46DB65F88CFC
:1002400011AF32CA57E97400000000240027002AC9
:1002500000524542000000000800020100000304B3
:10026000070000000000000000000000002300263E
:1002700000290000000000250028002B00040404D1
:10028000040404040402020202020203030303033F
:10029000030102040810204080010204081020011C
:1002A000020408102000F626302C11241FBECFEFC8
:1002B000D8E0DEBFCDBF13E0A0E0B1E0E2E4F2E7BA
:1002C00002C005900D92AA31B107D9F726E0AAE144
:1002D000B3E001C01D92A931B207E1F711E0C4E516
:1002E000D1E004C02197FE010E949135C335D107AA
:1002F000C9F70E947D280C9414390C9400000895CD
:1003000008950895AF92BF92CF92DF92EF92FF923D
:100310000F931F93CF93DF936C017B018B01040F2D
:10032000151FEB015E01AE18BF08C017D10759F0C9
:100330006991D601ED91FC910190F081E02DC6010B
:100340000995892B79F7C501DF91CF911F910F9105
:10035000FF90EF90DF90CF90BF90AF900895CF9334
:10036000DF93FC01448155816081718184E694E0D2
:100370000E948201EC0142E050E06BE571E084E60E
:1003800094E00E9482018C0F9D1FDF91CF91089510
:10039000FC01538D448D252F30E0842F90E0821B8B
:1003A000930B541710F0CF96089501970895FC0110
:1003B000918D828D981761F0A28DAE0FBF2FB11D68
:1003C0005D968C91928D9F5F9F73928F90E00895C0
:1003D0008FEF9FEF0895FC01918D828D981731F07A
:1003E000828DE80FF11D858D90E008958FEF9FEFCE
:1003F0000895FC01918D228D892F90E0805C9F4FA4
:10040000821B91098F739927089584E694E00E94D6
:10041000F90121E0892B09F420E0822F089580E082
:1004200090E0892B29F00E94050281110C940000B4
:100430000895FC01A48DA80FB92FB11DA35ABF4F79
:100440002C91848D90E001968F739927848FA689D3
:10045000B7892C93A089B1898C91837080648C9327
:10046000938D848D981306C00288F389E02D8081D6
:100470008F7D80830895EF92FF920F931F93CF9308
:10048000DF93EC0181E0888F9B8D8C8D98131AC0CF
:10049000E889F989808185FF15C09FB7F894EE89B6
:1004A000FF896083E889F989808183708064808313
:1004B0009FBF81E090E0DF91CF911F910F91FF905E
:1004C000EF900895F62E0B8D10E00F5F1F4F0F7306
:1004D0001127E02E8C8D8E110CC00FB607FCFACFC1
:1004E000E889F989808185FFF5CFCE010E94190244
:1004F000F1CFEB8DEC0FFD2FF11DE35AFF4FF08292
:100500009FB7F8940B8FEA89FB8980818062CFCFF7
:10051000CF93DF93EC01888D8823B9F0AA89BB893A
:10052000E889F9898C9185FD03C0808186FD0DC025
:100530000FB607FCF7CF8C9185FFF2CF808185FF46
:10054000EDCFCE010E941902E9CFDF91CF9108953E
:10055000833081F028F4813099F08230A9F0089539
:100560008730A9F08830C9F08430B1F480918000E0
:100570008F7D03C0809180008F77809380000895E5
:1005800084B58F7784BD089584B58F7DFBCF80912E
:10059000B0008F778093B00008958091B0008F7D78
:1005A000F9CFCF93DF93E4E6F2E08491E0EAF2E062
:1005B000D491ECE8F2E0C491CC23A1F081110E9427
:1005C000A802EC2FF0E0EE0FFF1FE759FD4FA591B9
:1005D000B491EC91ED2381E090E009F480E0DF91AB
:1005E000CF91089580E090E0FACF1F93CF93DF93EF
:1005F000282F30E0F901EB5AFD4F8491F901EF56B5
:10060000FD4FD491F901E358FD4FC491CC23A9F0DB
:10061000162F81110E94A802EC2FF0E0EE0FFF1FB1
:10062000ED58FD4FA591B4918FB7F894EC9111114D
:1006300008C0D095DE23DC938FBFDF91CF911F914F
:100640000895DE2BF8CFCF93DF9390E0FC01EF56B7
:10065000FD4F249183589D4FFC0184918823D1F054
:1006600090E0880F991FFC01E95BFD4FA591B491C3
:10067000FC01ED58FD4FC591D49161110EC09FB79B
:10068000F8948C91E22FE0958E238C932881E223BD
:10069000E8839FBFDF91CF9108958FB7F894EC91D5
:1006A000E22BEC938FBFF6CF8E3008F08E50209166
:1006B000060190E4299F900111248770822B80937A
:1006C0007C0080917A00806480937A0080917A0027
:1006D00086FDFCCF809178009091790008953FB716
:1006E000F8948091DA039091DB03A091DC03B09140
:1006F000DD0326B5A89B05C02F3F19F00196A11D6B
:10070000B11D3FBFBA2FA92F982F8827BC01CD015B
:10071000620F711D811D911D42E0660F771F881FBA
:10072000991F4A95D1F708958F929F92AF92BF92E9
:10073000CF92DF92EF92FF926B017C010E946F03D8
:100740004B015C01C114D104E104F104B9F00E9431
:100750006F03681979098A099B09683E734081050E
:10076000910580F321E0C21AD108E108F10888EE72
:10077000880E83E0981EA11CB11CE4CFFF90EF907F
:10078000DF90CF90BF90AF909F908F9008958F9201
:100790009F92AF92BF92EF92FF921F93CF93DF93FE
:1007A000C82F10920D0610920E0610920F0610928E
:1007B00010061092110661E08FE00E94230360E0B2
:1007C0008FE00E94F5026C2F70E090E080E00E94C4
:1007D000940360E08FE00E9423038BE990E001978F
:1007E000F1F7C0E9D1E00E94D102892B71F4219781
:1007F000D1F78EEF9FEFDF91CF911F91FF90EF9098
:10080000BF90AF909F908F900895C0E9D1E00E9473
:10081000D102019719F42197D1F7EBCFD8E2C0E8C4
:1008200010E090E9E92EFF24F3940E94D102892B75
:1008300029F481E0E81AF108C1F7DBCF0E946F03C9
:100840004B015C0180E9E82EFF24F3940E94D10261
:10085000019729F481E0E81AF108C1F7CACF0E9494
:100860006F03681979098A099B0969327105810545
:10087000910538F0E12FF0E0EB5FF94F80858C2B8C
:100880008087C69511F41F5FC0E8D15051F690E003
:1008900080E0B1CF8F929F92AF92BF92CF92DF92C2
:1008A000EF92FF920F931F93CF93DF938AE0A82ECE
:1008B000B12CD0E0C0E0EE24EA9493E0F92E882435
:1008C0008A9423E0922ED12CC12C10E000E08FE01E
:1008D0000E9454030817190790F1C816D90608F4A6
:1008E0006C018815990568F18E159F0508F47C0147
:1008F000C80FD91F65E070E080E090E00E9494038B
:1009000081E0A81AB10819F70C0D1D1DCE01801B3E
:10091000910B8E199F098819990966E070E00E9471
:100920006935CB01DF91CF911F910F91FF90EF902F
:10093000DF90CF90BF90AF909F908F9008958C01E3
:10094000D0CF4C01D5CF2FB7F8946091D6037091DA
:10095000D7038091D8039091D9032FBF0895DC016C
:1009600080E0615090F09D919827E92FEF70F0E0C2
:10097000E95DFD4F2491E92FE295EF70F0E0E95C2D
:10098000FD4FE491822F8E27ECCF0895DC012C914E
:100990001196ED91FC91F8948181822B8183928153
:1009A000322F30959323928387E090E00197F1F7FF
:1009B00081818323818383E290E00197F1F7908125
:1009C0007894EFECF0E03197F1F7922381E009F4AD
:1009D00080E00895FC0190810180F281E02D292FB3
:1009E000209560FF14C0F8948281822382838181E4
:1009F000892B8183A3E2B0E01197F1F78281982BD4
:100A00009283789487ED90E00197F1F70895F89438
:100A10008281822382838181892B8183AFEFB0E041
:100A20001197F1F78281982B928378948FE090E070
:100A3000EBCFDF92EF92FF920F931F93CF93DF9351
:100A4000EC01D62EE42E08E010E0FF24F39461E0E0
:100A50008D2D8F2109F460E0CE010E94EA04FF0C85
:100A600001501109A1F7E11010C0F894E981FA8151
:100A700091818881809589238183E981FA8192819E
:100A800088818095892382837894DF91CF911F910B
:100A90000F91FF90EF90DF900895EF92FF920F93E8
:100AA0001F93CF93DF938C017B0140E065E50E94AB
:100AB0001905E70188E0E80EF11C699140E0C801E2
:100AC0000E941905CE15DF05C1F7DF91CF911F9167
:100AD0000F91FF90EF900895FC0190810180F281C9
:100AE000E02DF8948181292F2095822381837894A9
:100AF0003DE743E050E0315029F1DA011197F1F779
:100B000080818923C1F3F894828182238283818149
:100B1000892B81837894ABE7B7E01197F1F7F894CC
:100B2000818182238183A3E1B1E01197F1F7808174
:100B3000982381E009F080E07894E3E6F6E03197CD
:100B4000F1F7089580E008956F927F928F929F92BF
:100B5000AF92BF92CF92DF92EF92FF920F931F93CB
:100B6000CF93DF93EC017B018A018E819F810E94EC
:100B70006C05811102C090E037C0B7018E819F8162
:100B80000E944D0540E06EEB8E819F810E94190509
:100B90007801680189E0C80ED11CAE80BF8088E072
:100BA000882E912C712C66246394C5010E94C60482
:100BB00081117628660CE1E08E1A9108B1F7F701F1
:100BC00071927F01EC15FD0541F78E819F810E9496
:100BD0006C05813081F668E0C8010E94AF0491E0A5
:100BE000F80120852813C7CF892FDF91CF911F915E
:100BF0000F91FF90EF90DF90CF90BF90AF909F90BC
:100C00008F907F906F900895CF93DF93CDB7DEB72D
:100C100029970FB6F894DEBF0FBECDBFAE014F5F70
:100C20005F4F0E94A405882331F08D818F33A9F096
:100C300020F48F31A1F080E007C08F3521F08F378D
:100C4000D1F78CE001C08BE029960FB6F894DEBF97
:100C50000FBECDBFDF91CF9108958AE0F5CF89E037
:100C6000F3CF2091F0033091F1032817390771F485
:100C70009091EE038091EF03981741F0E091EE031D
:100C8000F0E0EB56FC4F808190E008958FEF9FEFEE
:100C900008950895EF92FF920F931F93CF93DF93E0
:100CA000DC015C96ED90FC905D97E114F10479F421
:100CB00081E090E013969C938E93129790E080E0F1
:100CC000DF91CF911F910F91FF90EF900895519672
:100CD000ED91FC91529750968C915097982F90954A
:100CE0000FB75E962C915E97122F127021FD6095C2
:100CF000F8942081112319F1282B2083E7012197F3
:100D0000F1F728E0462F50E0308160FF1AC0382B01
:100D10003083E7012197F1F7BA0175956795215066
:100D200089F7112381F08081892380830FBF5C962E
:100D30008D919C910197F1F781E090E0C1CF29233B
:100D4000DCCF3923E5CF9081892BEFCF2091F003C1
:100D50003091F1032817390771F48091EF03209146
:100D6000EE0390E0805C9F4F821B910960E470E08D
:100D70000E947D35089590E080E008952091F00371
:100D80003091F10328173907B9F49091EE0380915F
:100D9000EF03981789F0E091EE03F0E0EB56FC4F7B
:100DA00080812091EE0330E02F5F3F4F2F73332778
:100DB0002093EE0390E008958FEF9FEF08950F9337
:100DC0001F930E94A3046093EE057093EF05809338
:100DD000F0059093F10586EE95E00E94BE0697FF20
:100DE0001DC00E94A3040091EE051091EF05209113
:100DF000F0053091F105601B710B820B930B009194
:100E0000EA051091EB052091EC053091ED05601796
:100E1000710782079307F8F28FEF9FEF1F910F91F1
:100E20000895E091F003F091F103E817F90769F4F0
:100E3000A389B4899C918589809589238C9310928C
:100E4000F1031092F00381E0089580E0089510927C
:100E50000106109200061092FF051092FE051092F6
:100E6000FD051092FC058DE991E0909303068093B7
:100E700002069091F205963108F046C02DEB30E065
:100E80003093FD052093FC052BE931E03093FF05FD
:100E90002093FE052CE231E03093010620930006FA
:100EA0002091680084E0983048F031E09E3008F4EA
:100EB00030E081E001C0880F3A95EAF7822B8093F9
:100EC00068002DE630E0983050F02BE630E09E30A0
:100ED00030F02CE630E0963110F030E020E0309336
:100EE000FA052093F905292F30E09830C0F581E00C
:100EF00001C0880F9A95EAF78093FB05809102065E
:100F0000909103060197F1F78091000690910106F8
:100F1000892B21F18091F0039091F10325E0863E29
:100F20009207E1F0009711F00E94110780910406EA
:100F30008E7F809304061092EF031092EE0386EEEC
:100F400095E09093F1038093F003E091F905F0911F
:100F5000FA0580819091FB05892B808308959E304E
:100F600040F42850310981E001C0880F2A95EAF742
:100F7000C3CF2E503109F7CF20917203260F3327AC
:100F8000331F21323105ECF420913A04FC0190E04A
:100F900080E0243069F082E00895A09172032191ED
:100FA000AC014E5A5C4FA40FB52FB11D2C93019686
:100FB000861798F380917203680F6093720380E044
:100FC000089581E0089510923A0481E080933904F5
:100FD0001092140461E082E10E94F50261E083E175
:100FE0000E94F502E9EBF0E080818E7F80838081B2
:100FF0008D7F808388E48093B80085E48093BC0073
:1010000008951092F3031092F2031092410410928B
:1010100063040E94E3078FE791E09093ED038093D0
:10102000EC0380E891E09093EB038093EA0308954A
:10103000CF93DF9391E0909351038823B9F0C0914F
:10104000B800D091BA008091BC008A7B8093BC002C
:1010500060E082E10E94F50260E083E10E94F50217
:101060000E94E307D093BA00C093B800DF91CF91FC
:101070000895CF92DF92EF92FF920F931F93CF9339
:10108000DF93D091630481E0D13208F09CC0C0911D
:1010900062040E946F036B017C0180913A0481110C
:1010A0006CC082E080933A0481E0809339048FEF32
:1010B0008093380410923704D0933604A2E4B4E04D
:1010C000E6E1F4E080E0D8138DC010921504809121
:1010D0001504CC0FC82BC0931504809114048130E3
:1010E00009F084C0109214040E946F036B017C010C
:1010F000809115048093BB0080913C0490913D0445
:10110000A0913E04B0913F04892B8A2B8B2BA1F038
:101110000E946F0300913C0410913D0420913E0415
:1011200030913F046C197D098E099F090617170736
:101130002807390708F442C08091BC0083FDD8CF4E
:1011400085EC8093BC000E946F036B017C01809151
:101150003A04823009F44CC0809138048F3F09F47E
:1011600069C080913804803209F466C080913804E7
:10117000803309F463C084E026C080913C049091E0
:101180003D04A0913E04B0913F04892B8A2B8B2B08
:1011900009F483CF0E946F0300913C0410913D0439
:1011A00020913E0430913F046C197D098E099F09FE
:1011B000061717072807390708F06FCF80913B04FF
:1011C0000E94180885E01092410410926304109266
:1011D0004004DF91CF911F910F91FF90EF90DF902E
:1011E000CF9008959D9191938F5F6DCF85EEA9CF9C
:1011F00080913C0490913D04A0913E04B0913F0445
:10120000892B8A2B8B2B09F4A2CF0E946F030091AC
:101210003C0410913D0420913E0430913F046C1930
:101220007D098E099F09061717072807390708F057
:101230008ECFC4CF80E0C7CF82E0C5CF83E0C3CFDD
:10124000CF92DF92EF92FF920F931F93CF93DF9392
:10125000D82FC62F613208F098C00E946F036B012F
:101260007C0180913A0481116BC081E080933A0443
:10127000809339049FEF90933804109237049C0FA9
:10128000909336048093150480911504DD0FD82BBC
:10129000D093150480911404813009F078C0109225
:1012A00014040E946F036B017C01809115048093EC
:1012B000BB0080913C0490913D04A0913E04B0910C
:1012C0003F04892B8A2B8B2BA1F00E946F03009186
:1012D0003C0410913D0420913E0430913F046C1970
:1012E0007D098E099F09061717072807390708F493
:1012F00048C08091BC0083FDD8CF85EC8093BC00B2
:101300000E946F036B017C0180913A04813009F4E3
:1013100040C0809137048C1710F4C0913704E6E187
:10132000F4E0A4EFB3E080E08C1355C08C2FDF9184
:10133000CF911F910F91FF90EF90DF90CF90089584
:1013400080913C0490913D04A0913E04B0913F04F3
:10135000892B8A2B8B2B09F484CF0E946F03009179
:101360003C0410913D0420913E0430913F046C19DF
:101370007D098E099F09061717072807390708F006
:1013800070CF80913B040E941808C0E0CFCF85EE5B
:10139000B5CF80913C0490913D04A0913E04B09162
:1013A0003F04892B8A2B8B2B09F4AECF0E946F034D
:1013B00000913C0410913D0420913E0430913F0483
:1013C0006C197D098E099F09061717072807390729
:1013D00008F09ACFD6CF91919D938F5FA5CFE091E2
:1013E000F3038091F203E81730F4F0E0EC50FC4F87
:1013F000808190E008958FEF9FEF08959091F3031F
:101400008091F2032FEF3FEF981748F4E92FF0E0B7
:10141000EC50FC4F208130E09F5F9093F303C901B3
:1014200008958091F2039091F303891B990B08951D
:10143000CF92DF92EF92FF920F931F93CF93DF93A0
:101440007C01CB018A0120914004222389F0EB0129
:101450006B01C40ED51ECC15DD0569F06991D7016D
:10146000ED91FC910190F081E02DC7010995F3CF3A
:10147000642F0E94BC07C801DF91CF911F910F918B
:10148000FF90EF90DF90CF900895CF93DF931F925E
:10149000CDB7DEB76983209140042223F9F0209173
:1014A0006304203258F021E030E0FC0133832283D2
:1014B00090E080E00F90DF91CF91089580914104FA
:1014C000E82FF0E0EE5BFB4F998190838F5F809374
:1014D00041048093630481E090E0ECCF61E0CE01B1
:1014E00001960E94BC07F7CF90E080E0089586EE59
:1014F00095E00E9411070C9427072F923F924F927C
:101500005F926F927F928F929F92AF92BF92CF9293
:10151000DF92EF92FF920F931F93CF93DF93CDB79C
:10152000DEB72D970FB6F894DEBF0FBECDBF1C01FE
:101530000E94770A64E670E080E090E00E949403E5
:101540006AE070E080E090E00E949403C101880F9F
:10155000991F9D878C87D12CC12CF12CE12C412C1B
:10156000512C320149E050E06CE171E086EE95E0EB
:101570000E94820165E070E080E090E00E949403A8
:1015800010E000E0812C912C540186EE95E00E9441
:10159000A606892B39F4F4E08F169104A104B10456
:1015A0000CF05FC0023011050CF05BC086EE95E0D8
:1015B0000E94A606892B99F086EE95E00E94BE0651
:1015C000E1E0F0E0EC0FFD1FE00FF11F80836AE027
:1015D00070E080E090E00E9494030F5F1F4F65E091
:1015E00070E080E090E00E9494030230110509F061
:1015F00070C089818F3F09F06CC08A81863809F0FC
:1016000068C0FE013396FB87EA8786EE95E00E946C
:10161000A606892B39F4F4E08F169104A104B104D5
:101620000CF050C00930110509F059C08B8190E0D1
:10163000982F88272C81820F911D092E000CAA0B50
:10164000BB0B480E591E6A1E7B1E40C0EC85FD85F3
:10165000EC15FD0509F086CFE114F10441F47101A8
:1016600006C08FEFC81AD80AE214F3047CF3C30152
:10167000B2010E94B0304B015C01B701FF0C880B36
:10168000990B0E94B0309B01AC01C501B4010E94CE
:10169000CE322D960FB6F894DEBF0FBECDBFDF91D0
:1016A000CF911F910F91FF90EF90DF90CF90BF905F
:1016B000AF909F908F907F906F905F904F903F90F2
:1016C0002F900895043011050CF0B0CFFFEFEF1A02
:1016D000FF0A8FEF881A980AA80AB80A56CF86EE32
:1016E00095E00E94BE06EA85FB858193FB87EA8729
:1016F0000F5F1F4F8ACF8F929F92AF92BF92CF9270
:10170000DF92EF92FF92CF93DF93C8EBD5E0988101
:1017100021E02093400490936204109241041092BF
:101720006304682F81E095E00E94450A0E94390811
:1017300063E088810E9420091092F3038093F203F2
:1017400081E095E00E94FE09092E000CAA0BBB0B5C
:101750008824982EA92EBA2E81E095E00E94FE09D9
:10176000092E000CAA0BBB0B6C017D01C828D928DF
:10177000EA28FB28FE2CED2CDC2CCC2481E095E023
:101780000E94FE09BC01990F880B990B6C297D29D9
:101790008E299F29DF91CF91FF90EF90DF90CF901E
:1017A000BF90AF909F908F9008958F929F92AF922D
:1017B000BF92CF92DF92EF92FF920F931F932091EF
:1017C000C1052F3F19F48AEF0E947B0B0091C505DC
:1017D0001091C60530E020E0C72ED82EE92EFF2458
:1017E000E7FCFA94C01AD10AE20AF30A57E0959589
:1017F0008795779567955A95D1F7000F111F221F8E
:10180000331F4B015C01801A910AA20AB30AA50199
:101810009401A091C705B091C8050E94F1314B0118
:101820005C01FBE0B594A79497948794FA95D1F75F
:10183000A7019601C701B6010E9459359B01AC0171
:10184000ACE05595479537952795AA95D1F7A09186
:10185000C905B091CA050E94F1319B01AC01BEE0FF
:101860005595479537952795BA95D1F7280D391D88
:101870004A1D5B1D2093BD053093BE054093BF05F7
:101880005093C005A5E0B0E00E94E63160587F4F5C
:101890008F4F9F4F672F782F892F992787FD9A9514
:1018A0000E94B03020E030E048EC52E40E94CE329A
:1018B0001F910F91FF90EF90DF90CF90BF90AF906E
:1018C0009F908F9008952F923F924F925F926F92C8
:1018D0007F928F929F92AF92BF92CF92DF92EF92C0
:1018E000FF920F931F93CF93DF93CDB7DEB76B9724
:1018F0000FB6F894DEBF0FBECDBF0E94D50B80910E
:10190000C1058F3F39F487EF0E947B0B6E8B7F8B75
:10191000888F998F8091BD059091BE05A091BF05DC
:10192000B091C0056C017D01FF0CCC08DC2C760168
:101930009C01AD016C2D7C2D8C2D9C2D345F414084
:101940005109610971098109910929873A874B87F2
:10195000652E762E872E982E9B8F5901C42ED52E5C
:10196000E62EF72E082F192F0E949735322E232EA0
:10197000488B598B6A8B7B8B8C8B9D8B3091CE05E2
:101980002091CD05932F990F990B492F592F692F2E
:10199000792F892F0E9497350CE00E948F3629837A
:1019A0003C874A8F5D876E877F87582E492E3091FE
:1019B000D0052091CF05932F990F990BA32CB22C12
:1019C000C888D988EA88FB880C891D89492F592F36
:1019D000692F792F892F0E94973508E00E94A83639
:1019E000A980BC84CA8CDD84EE84FF84052D142D6F
:1019F0000E94C53670588F4F9F4FE091CB05F091F4
:101A0000CC055F01D12CC12CE12CF12C8701E9839D
:101A1000BA82CB82DC82ED82FE820F831887C12CD2
:101A2000D12CE12CF12C00E010E00E94973501E26E
:101A30000E94A8362A8F532E49835C876D877E8744
:101A40008F87492EA0E00E94D73609F436C1309125
:101A5000D6052091D505932F990F990BA32CB22C65
:101A6000C888D988EA88FB880C891D89492F592F95
:101A7000692F792F892F0E9497351901488B598B2F
:101A80006A8B7B8B8C8B9D8B3091D4052091D305F9
:101A9000932F990F990BA984BA84CB84D62CE72C69
:101AA000F82C092D1B8D492F592F692F792F892F3C
:101AB0000E94973501E10E948F365101C888D9886C
:101AC000EA88FB880C891D890E94C53659016A0184
:101AD0007B01382E192F4E895F89688D798D84E0BE
:101AE00075956795579547958A95D1F780E090E071
:101AF000A0E1B0E0841B950BA60BB70B3C014D0198
:101B0000990C6608762C43019C01AD01662D762D5B
:101B1000862D962D0FE10E948F36722E832E942EE5
:101B20005987B62FA72FF82FE92F3091D205209192
:101B3000D105932F990F990B492F592F692F792F81
:101B4000892F03E20E948F36032D0E94C53659016A
:101B50006A017B018C01272D382D492D59856B2F6A
:101B60007A2F8F2F9E2F0E94CE36E5E3AE2EFCE01B
:101B7000BF2EC12CD12CE12CF12C00E010E00E94F2
:101B80009735AA8CB52CC980DC84ED84FE840F8542
:101B9000142D0E94F1352F873E8749875A876B871E
:101BA00079838C879D870DE00E94A836922E832E24
:101BB000742E652E562E472E382E292E3091DC0598
:101BC0002091DB05932F990F990BA92CB82CC72CCA
:101BD000D62CE52CF42C032D122D492F592F692FCB
:101BE000792F892F0E9497350E94973509E10E942D
:101BF000A836AF84BE84C984DA84EB84F9800C856E
:101C00001D850E94C53619012A013B014C01309106
:101C1000DA052091D905932F990F990B492F592F48
:101C2000692F792F892F0E94973503E10E94A836EA
:101C300059016A017B018C019101A201B301C40128
:101C40000E94C53608E00E94A83659016A017B014E
:101C5000E82F192F3091D8052091D705932F990F90
:101C6000990B492F592F692F792F892F04E00E9452
:101C70008F360E2F0E94C5360E94763320E030E06A
:101C800040E85BE30E940F316B960FB6F894DEBF1D
:101C90000FBECDBFDF91CF911F910F91FF90EF90BD
:101CA000DF90CF90BF90AF909F908F907F906F907C
:101CB0005F904F903F902F90089560E070E0CB01CF
:101CC000E3CFBF92CF92DF92EF92FF920F931F93D9
:101CD000CF93DF93EC01B62EC72E8D85811105C001
:101CE000CE010E946C0581110EC01B861D861C86CC
:101CF00080E0DF91CF911F910F91FF90EF90DF90E7
:101D0000CF90BF90089540E060EFCE010E9419058A
:101D100001E0E12CD12C11E0CE010E94C604F82E86
:101D2000CE010E94C60491E0F91218C0813099F5E5
:101D30001134D8F2DB86D11002C081E08D878B810F
:101D4000882399F22396EB2DFC2DCF01089629913B
:101D50002193E817F907D9F781E0CBCFEE2DF0E01A
:101D6000F8120FC08B851817A0F4DE01AE0FBF1F4D
:101D700013968C91802379F4F12C193008F41C8788
:101D8000D12EEC0FFD1F8381902F909589238383A3
:101D90000AC08113F1CFFE01EE0DF11D8381802B6E
:101DA0008383FF24F3946F2DCE010E94EA041F5F0A
:101DB000000F11F4E39401E087E08E1508F0ACCF3A
:101DC000B7CFDF92EF92FF920F931F93CF93DF93E2
:101DD0007C018B01D42EDC011696ED91FC911386CB
:101DE0001586148612861186108617821682158231
:101DF00014821382C0E0B801F701868197810E94A6
:101E0000610ED82F882329F0DC1629F0CF5FDC166D
:101E100090F7D0E009C067E0C8010E94AF04D80184
:101E200017969C918913F2CF8D2FDF91CF911F913F
:101E30000F91FF90EF90DF900895CF939091C1059F
:101E40009F3F41F5682F8091B80591E09093400441
:101E500080936204109241041092630481E095E043
:101E60000E94450A0E94390862E08091B8050E94EC
:101E700020091092F3038093F20381E095E00E9421
:101E8000FE09C82F81E095E00E94FE0920E03C2F6A
:101E9000282B392B922F832FCF9108950F931F93C7
:101EA000CF93DF93FC01048115810115110539F4ED
:101EB000FB011082DF91CF911F910F910895415046
:101EC00051094017510708F48A01EB01FC016081B8
:101ED0007181A801CE010E94EB38C00FD11F18827A
:101EE000E9CFCF93DF93C091AC05D091AD0520979A
:101EF00061F08991882349F0082E000C990B0E940B
:101F0000C538FE0131978083F4CFDF91CF910895DA
:101F100085ED8093BC0080913C0490913D04A0919C
:101F20003E04B0913F040796A11DB11D23E0B69574
:101F3000A795979587952A95D1F72091BC0024FD08
:101F400003C010923A04089540913C0450913D041E
:101F500060913E0470913F04452B462B472B69F35B
:101F60000097A105B10541F025E32A95F1F700009E
:101F70000197A109B109E1CF80913B040C941808A5
:101F8000FC0180819181009711F00C94802C60E01D
:101F900070E0CB010895AF92BF92CF92DF92EF92A3
:101FA000FF920F931F93CF93DF93DC01CD90DC90D2
:101FB0001197C114D10439F01496CD91DC918C01A4
:101FC0007601209761F4DF91CF911F910F91FF90DF
:101FD000EF90DF90CF90BF90AF90089575015701BB
:101FE000BFEFAB1ABB0AF7018081082E000C990BDA
:101FF0000E947830892B91F72197CC0DDD1D8881C7
:10200000082E000C990B0E947830892B29F0CE15F0
:10201000DF0510F02197F3CFAE014F5F5F4F4E19F0
:102020005F09D80115965C934E931497CE14DF0484
:1020300020F4B701C6010E94CD38D801ED91FC9182
:10204000119714968D919C91E80FF91F1082BBCFC8
:10205000FB0144815581FC0124813581241735071A
:1020600078F080819181009759F0FB016081718146
:102070006115710529F00E94DD3821E0892B09F0F6
:1020800020E0822F08950F931F93CF93DF938C014D
:10209000EB01FC01808191810097E1F068817981F9
:1020A00061157105A9F0428153812C813D81421750
:1020B000530770F00E94D6388C819D81F80195837A
:1020C00084831D821C82DF91CF911F910F9108950F
:1020D0000E947F3788819981F801918380838A816A
:1020E0009B81938382838C819D81958384831982D4
:1020F00018821B821A82E5CFCF93DF93EC0188818F
:102100009981009711F00E947F37198218821D82F1
:102110001C821B821A82DF91CF910895FC0180817D
:102120009181009711F00C947F3708950F931F93BE
:10213000CF93DF93EC0188819981009759F02A8130
:102140003B812617370730F081E0DF91CF911F9157
:102150000F9108958B016F5F7F4F0E9408380097A1
:1021600059F0998388831B830A832C813D81232B1B
:1021700059F7FC011082E8CF80E0E7CFEF92FF92A1
:102180000F931F93CF93DF936115710541F480E0A6
:10219000DF91CF911F910F91FF90EF90089541151E
:1021A0005105B1F07B01EC010C811D81040F151F5D
:1021B000B8010E949610882351F3288139818C81BF
:1021C0009D81B701820F931F0E94D6381D830C8317
:1021D00081E0DECFFC01448155816081718182EB19
:1021E00095E00C94BE100F931F93CF93DF9300D014
:1021F000CDB7DEB78C0119821A8241E050E0BE01F2
:102200006F5F7F4F0E94BE10811103C0C8010E9402
:102210007C10C8010F900F90DF91CF911F910F910B
:102220000895CF93DF93EC01FB0101900020E9F7C3
:102230003197AF01461B570B0E94BE10811103C09E
:10224000CE010E947C10CE01DF91CF910895CF93F3
:10225000DF93EC01FB0144815581608171810E9413
:10226000BE10811103C0CE010E947C10CE01DF910F
:10227000CF910895EF92FF920F931F93CF93DF9327
:10228000EC018B01CB010E94AE2C7C01BC01CE0184
:102290000E94961081110BC0CE010E947C10CE01CD
:1022A000DF91CF911F910F91FF90EF900895FD82E4
:1022B000EC82B801888199810E94A72CF0CFEF921F
:1022C000FF920F931F93CF93DF93EC017B018A0161
:1022D000BA010E94961081110BC0CE010E947C10A1
:1022E000CE01DF91CF911F910F91FF90EF90089554
:1022F0001D830C83B701888199810E94D638F0CF65
:10230000FB0101900020E9F73197AF01461B570B05
:102310000C945F110F931F93CF93DF93CDB7DEB76C
:1023200062970FB6F894DEBF0FBECDBF8C01CB0114
:10233000F8011182108213821282158214824AE0FF
:10234000BE016F5F7F4F0E94B72CBE016F5F7F4F52
:10235000C8010E94801162960FB6F894DEBF0FBECE
:10236000CDBFDF91CF911F910F910895CF93DF9350
:10237000EC01FB018617970749F0608171816115B7
:10238000710541F0448155810E945F11CE01DF91BA
:10239000CF9108950E947C10F9CFFC011182108228
:1023A00013821282158214820C94B611FC011182E0
:1023B00010821382128215821482FB010190002088
:1023C000E9F73197AF01461B570B0C945F11AF92A1
:1023D000BF92CF92DF92EF92FF920F931F93CF9312
:1023E000DF936C015B017A0189012417350720F422
:1023F0008F2D7901042F182F6DE571E0C6010E9421
:10240000D611D5011496CD91DC91EC16FD06E0F4C1
:102410000C171D0708F4E801D501ED91FC91119707
:10242000EC0FFD1F108110826D917C916E0D7F1D50
:10243000C60161157105A1F00E948011F50180812E
:102440009181C80FD91F1883C601DF91CF911F91C9
:102450000F91FF90EF90DF90CF90BF90AF900895D5
:102460000E947C10EBCFCF93DF93EC01FB01248122
:1024700035810E94E711CE01DF91CF9108950F932E
:102480001F93CF93DF93CDB7DEB72C970FB6F89499
:10249000DEBF0FBECDBFFC012481358112161306AD
:1024A00064F48C01253131059CF40E94AF0164E194
:1024B00070E080E090E00E9494032C960FB6F894B0
:1024C000DEBF0FBECDBFDF91CF911F910F91089559
:1024D0002FE030E050E040E0BC01CE0107960E94C2
:1024E000E7114B855C856F81788584E694E00E94D6
:1024F000820169E170E080E090E00E9494034FE087
:1025000050E0B801CE0101960E943312BE016F5F08
:102510007F4FCE0107960E944310CE0101960E9484
:102520008E10CE0107960E94AF0164E170E080E05A
:1025300090E00E9494036DE571E0CE0107960E9441
:102540008011CE0107960E948E10B7CFEF92FF92B6
:102550000F931F93CF93DF93CDB7DEB7A1970FB63D
:10256000F894DEBF0FBECDBF7C01CB01BA01F701ED
:1025700011821082138212821582148242E0420F6D
:102580008E010F5F1F4F0E945E2C009789F0BC01E7
:10259000C7010E948011A1960FB6F894DEBF0FBE4E
:1025A000CDBFDF91CF911F910F91FF90EF900895D4
:1025B000C7010E947C10EFCFFF920F931F93CF9320
:1025C000DF93EC01F62E08811981C8010E94D031F9
:1025D000F81621F06F2DC8010E94D831CE01DF918D
:1025E000CF911F910F91FF900895EF92FF920F935B
:1025F0001F93CF93DF9300D0CDB7DEB70DE015E08A
:102600008D5095407C01C701800F911F9A8389836B
:10261000F80161918F01CE0101960E94DC12F5E074
:102620000B351F0781F78DE095E00F900F90DF913C
:10263000CF911F910F91FF90EF900895EF92FF922D
:102640000F931F93CF93DF9300D0CDB7DEB701E692
:1026500015E0815695407C01C701800F911F9A8338
:102660008983F80161918F01CE0101960E94DC12ED
:10267000F5E008381F0781F781E695E00F900F908D
:10268000DF91CF911F910F91FF90EF9008954F929E
:102690005F926F927F928F929F92AF92BF92CF92F2
:1026A000DF92EF92FF920F931F93CF93DF93CDB7FB
:1026B000DEB76E970FB6F894DEBF0FBECDBF1A829D
:1026C00019821C821B821E821D8263E272E0CE018F
:1026D00001960E943A11BE016F5F7F4F8CEA95E030
:1026E0000E942810182FCE0101960E948E101123EF
:1026F00011F16EE571E0CE0101960E94D61168E8F5
:1027000075E0CE0101960E942711BC0182EB95E095
:102710000E94B611CE0101960E948E1062EB75E008
:10272000CE0101960E94CD11CE0101960E943F126A
:10273000CE010196EAC31A8219821C821B821E8274
:102740001D826FE172E0CE0101960E943A11BE0136
:102750006F5F7F4F8CEA95E00E942810182FCE0102
:1027600001960E948E10112359F068E671E082EB09
:1027700095E00E9480118EE895E00E94EA10CECF8D
:1027800066E771E0CE0101960E94D611BE016F5F2F
:102790007F4F8CEA95E00E942810182FCE010196F9
:1027A0000E948E101123C9F127E030E046E050E08E
:1027B00060EA75E0CE0101960E94E711BE016F5FED
:1027C0007F4F8AE995E00E944310CE0101960E9456
:1027D0008E108AE995E00E94C00F672B21F41092B9
:1027E000E00381E003C081E08093E0036E960FB6C2
:1027F000F894DEBF0FBECDBFDF91CF911F910F9137
:10280000FF90EF90DF90CF90BF90AF909F908F9010
:102810007F906F905F904F9008956DE771E0CE01CB
:1028200001960E94D611BE016F5F7F4F8CEA95E042
:102830000E942810182FCE0101960E948E1011239D
:1028400009F4B5C080914F039091500318161906F2
:1028500044F688EC90E0909305018093040184E6AF
:1028600094E00E9488021D861E861F86188ACC244A
:10287000C394D12C60EC462E63E0562E5E012DE011
:10288000A20EB11C3E0131E1630E711C80914F0319
:10289000909150038C159D050CF4A3CF80910401F9
:1028A00090910501813C934024F0509205014092A3
:1028B00004010091040110910501750148018A1875
:1028C0009B08C4018E0D9F1D0E94D031F70181939A
:1028D0007F01E615F705A9F7C80104969093050155
:1028E000809304014BE2E42E43E0F42E07521340A0
:1028F000C8018E0D9F1D0E94D031F70181937F0189
:10290000FFE4EF16F3E0FF0699F74D855E856F85CE
:10291000788923E0CE0107960E94A612BE01695F66
:102920007F4FCE0101960E94CD1161E871E0CE018A
:1029300001960E941111BC0182EB95E00E94B61134
:10294000CE0101960E948E10CE0107960E948E1035
:102950006BE273E0CE0101960E94D611CE01019682
:102960000E94EA10CE0101960E948E1062EB75E083
:10297000CE0101960E94CD11CE0101960E943F1218
:10298000CE0101960E948E10809104019091050164
:102990008496909305018093040164E170E080E0E7
:1029A00090E00E9494032FEFC21AD20A6FCF64E81E
:1029B00071E0CE0101960E94D611BE016F5F7F4F7C
:1029C0008CEA95E00E942810182FCE0101960E94F3
:1029D0008E101123F1F126E030E045E050E060EA8E
:1029E00075E0CE0101960E94E711BE016F5F7F4F37
:1029F0008AE995E00E944310CE0101960E948E1054
:102A00008AE995E00E94C00F672B19F410922A03FF
:102A1000E8CE81E080932A0388EC90E09093050152
:102A2000809304011092500310924F0310922603DA
:102A30001092270310922803109229030E94A304E6
:102A400060932203709323038093240390932503C0
:102A5000C8CE6AE871E0CE0101960E94D611BE018F
:102A60006F5F7F4F8CEA95E00E942810182FCE01EF
:102A700001960E948E10112309F476C08091A4055E
:102A80009091A505079708F4ACCE46E050E060EAC7
:102A900075E0CE0101960E943312BE016F5F7F4F39
:102AA0008AE995E00E944310CE0101960E948E10A3
:102AB00080919A0590919B05C12CD12C76010097AD
:102AC00021F00E947C2C6B017C01C0920C01D09201
:102AD0000D01E0920E01F0920F0161E971E082EBCD
:102AE00095E00E94801122E0B701A601CE01079671
:102AF0000E94A612BE01695F7F4FCE0101960E941F
:102B0000CD1169EB72E0CE0101960E9411110E9475
:102B1000EA10CE0101960E948E10CE0107960E9407
:102B20008E1062EB75E0CE0101960E94CD11CE01B0
:102B300001960E943F12CE0101960E948E100E94C3
:102B4000A30428EE33E040E050E00E943032CA0196
:102B5000B9010E94AE306093E5037093E603809361
:102B6000E7039093E8033DCE6CE971E0CE01019656
:102B70000E94D611BE016F5F7F4F8CEA95E00E94E4
:102B80002810182FCE0101960E948E10112309F4EF
:102B900054C08091A4059091A505079708F421CE13
:102BA00046E050E060EA75E0CE0101960E943312E3
:102BB000BE016F5F7F4F8AE995E00E944310CE010E
:102BC00001960E948E1080919A0590919B05C12CD0
:102BD000D12C7601009721F00E947C2C6B017C01A6
:102BE000C0920001D0920101E0920201F092030133
:102BF00063EA71E082EB95E00E94801121E0B70169
:102C0000A601CE0107960E94A612BE01695F7F4F02
:102C1000CE0101960E94CD1169EB72E0CE010196C2
:102C20000E9411110E94EA10CE0101960E948E109E
:102C3000CE0107960E948E1071CD6EEA71E0CE0132
:102C400001960E94D611BE016F5F7F4F8CEA95E01E
:102C50000E942810182FCE0101960E948E10112379
:102C600041F126E030E044E050E060EA75E0CE015A
:102C700001960E94E711BE016F5F7F4F8AE995E0E0
:102C80000E944310CE0101960E948E108AE995E0C1
:102C90000E94C00F70930E0560930D05709309019B
:102CA0006093080180910A0190910B010E94F51236
:102CB00098CD63EB71E0CE0101960E94D611BE0162
:102CC0006F5F7F4F8CEA95E00E942810182FCE018D
:102CD00001960E948E101123A9F143E050E060EAB2
:102CE00075E0CE0101960E943312BE016F5F7F4FE7
:102CF0008AE995E00E944310CE0101960E948E1051
:102D00006AE975E0CE0101960E94CD11CE010196CF
:102D10000E94F310BC018EE895E00E94B611CE012E
:102D200001960E948E104091920550919305411595
:102D3000510509F4B7CF6FE075E08EE895E00E9489
:102D40004E0FB0CF6AEB71E0CE0101960E94D61112
:102D5000BE016F5F7F4F8CEA95E00E942810182F0C
:102D6000CE0101960E948E10112309F482C0809139
:102D7000A4059091A505409708F0DAC242E050E022
:102D800060EA75E0CE0101960E943312BE016F5FCA
:102D90007F4F8AE995E00E944310CE0101960E9480
:102DA0008E1080919A0590919B050097F1F10E94F9
:102DB0007C2C20E030E048EC52E40E940F310E946D
:102DC00040336093190570931A0580931B05909307
:102DD0001C0567EB71E082EB95E00E948011609129
:102DE000190570911A0580911B0590911C058B01A6
:102DF0009C0100591F452140310901341C4921051E
:102E00003105B8F06AE975E0CE0101960E94CD1156
:102E10006DEB71E0CE0101960E9411110E94EA1043
:102E2000CE0101960E948E10DCCC60E070E0CB01F8
:102E3000C0CF0E94B03020E030E048EC52E40E9465
:102E4000CE32AB01BC0122E0CE0101960E94A61257
:102E5000CE0101960E94EA10CE0101960E948E10CA
:102E600043E050E06AEC71E082EB95E00E94BE1016
:102E700019CF6EEC71E0CE0101960E94D611BE0111
:102E80006F5F7F4F8CEA95E00E942810182FCE01CB
:102E900001960E948E101123D9F1809159059091CD
:102EA0005A05019709F09DCC6DE571E0CE010D96B4
:102EB0000E94D61189899A89009729F1ED85FE85AE
:102EC0002081222301F10797F0F064ED71E0CE013B
:102ED00007960E94D611BE01635F7F4FCE01079611
:102EE0000E942711BC01CE0101960E94CD11CE0196
:102EF00001960E943F12CE0101960E948E10CE01D3
:102F000007960E948E10CE010D960E948E1069CCFD
:102F100069ED71E0CE0101960E94D611BE016F5F8E
:102F20007F4F8CEA95E00E942810182FCE01019661
:102F30000E948E101123F1F025E030E044E050E0D3
:102F400060EA75E0CE0101960E94E711BE016F5F55
:102F50007F4F8AE995E00E944310CE0101960E94BE
:102F60008E108AE995E00E94C00F70935A05609315
:102F7000590598CE6EED71E0CE0101960E94D611F2
:102F8000BE016F5F7F4F8CEA95E00E942810182FDA
:102F9000CE0101960E948E10112309F45EC009E152
:102FA00010E0C12CD12C760180E10E945403BC01B9
:102FB000990F880B990B0E94B0309B01AC01C7019F
:102FC000B6010E9462326B017C016AE070E080E031
:102FD00090E00E9494030150110931F720E030E0A5
:102FE00040EA50E4C701B6010E940F3120E030EC06
:102FF0004FE754E40E94CE3220E030E048EC51E448
:103000000E94CE3260933505709336058093370564
:103010009093380580910A0190910B010E94F5125E
:1030200062EE71E082EB95E00E94801140913505DF
:1030300050913605609137057091380522E0CE0138
:1030400007960E94A612BE01695F7F4FCE010196CE
:103050000E94CD116AEE71E0E1CD6DEE71E0CE011E
:1030600001960E94D611BE016F5F7F4F8CEA95E0FA
:103070000E942810182FCE0101960E948E10112355
:1030800009F4AFCB43E050E06CEA75E0CE0107965F
:103090000E943312BE01695F7F4FCE0101960E94EC
:1030A000CD11CE0101960E94F310BC018AE995E092
:1030B0000E94B611CE0101960E948E10CE01079695
:1030C0000E948E106AE975E0CE0149960E94CD11EA
:1030D00061EF71E0CE0101960E94D6118D8D9E8D1B
:1030E000892BC9F1098D1A8D69817A81C8010E94E5
:1030F000FA38009781F1FC01E01BF10B8F01CE0142
:1031000001960E948E106DE571E0CE0143960E94FB
:10311000D6116DE571E0CE010D960E94D611101604
:103120001106E4F463EF71E0CE0101960E94D6111E
:10313000CE0101960E943F12CE0101960E948E1090
:10314000CE010D960E948E10CE0143960E948E10E5
:10315000CE014996DACE0FEF1FEFD1CFBE01675EE9
:103160007F4FCE010D960E94B61110E000E02AEFCD
:10317000A22EBB24BA9436E0932E89899A890097AF
:1031800009F4C7C005301105D1F362ED71E0CE013D
:1031900001960E94D611BE016F5F7F4FCE010D9642
:1031A0000E942810F82ECE0101960E948E10F11078
:1031B000A0C0EE24E394F12C970150E040E0BE0162
:1031C000635F7F4FCE0107960E94E711BE01695FE2
:1031D0007F4FCE0101960E94CD11CE0101960E9433
:1031E000F310BC01CE0143960E94B611CE010196A8
:1031F0000E948E10CE0107960E948E10BE016D5E59
:103200007F4FCE0107960E94CD118B859C8502973A
:1032100008F473C062ED71E0CE0101960E94D611F0
:10322000BE016F5F7F4FCE0107960E942810D82EF7
:10323000CE0101960E948E10DD2009F45EC022E0CE
:1032400030E041E050E0BE01695F7F4FCE01019662
:103250000E94E711CE0101960E94C00F2B016B0165
:10326000CE0101960E948E1057FE03C0FCE1CF0EE6
:10327000D11CB5016C197D09909E6001919ED00C06
:103280001124F601EF59FA4F76876587CE0107962C
:103290000E948E10B60166597A4F44E050E0CE018C
:1032A00043960E944E0F0F5F1F4F89899A89E81637
:1032B000F90640F5A701BE01635F7F4FCE0101967D
:1032C0000E943312BE016F5F7F4FCE0143960E9472
:1032D0004310CE0101960E948E10BE016D5E7F4F9D
:1032E000CE010D960E94B611CE010D960E94CB0F15
:1032F00044CF82E0E82EF12C5FCFCE0107960E94EA
:10330000C00FBACF6DE571E0CE010D960E9480111D
:1033100034CF00936305002341F081E08093610581
:103320008EE190E00E941E130BCF10926105F8CF42
:1033300080E05CCA2F923F924F925F926F927F9291
:103340008F929F92AF92BF92CF92DF92EF92FF92B5
:103350000F931F93CF93DF93CDB7DEB7CD54D10931
:103360000FB6F894DEBF0FBECDBF7C016DE571E0F6
:1033700082EB95E00E948011C7010596059768F0E1
:103380008091E903811109C02CEEE2162FEFF206BD
:1033900024F0F092E403E092E303F7017A96E4323A
:1033A000F10510F00C948B24E852F64E0C949135F4
:1033B00018248B2414248B248B248B248B248B247F
:1033C0008B248B248B24A01CA01CA01CFC19A41DE6
:1033D000A01CA21E761FA01CA01CA820B720BA20EB
:1033E0008B24A01CA01CC82067225E23EF230A2484
:1033F000A01CA01CA01CA01C60E08FE00E94230366
:10340000E0EAF2E0E491E8A3ECE8F2E0E491F0E035
:10341000EE0FFF1FE759FD4F859194919AA389A361
:103420001BA61DA61CA6CE01809698878F831D82A1
:103430001E82198289E08A8381E08B838C831C8AB7
:103440001B8A1AA619A618A61FA21EA21DA21CA29C
:103450001BA201E0BE01625D7F4F8F8198850E94B3
:10346000610E882309F45CC067E0CE018E960E944D
:10347000AF049DA98913EECF898181111DC08F8171
:1034800098850E946C05BE01625D7F4F8F81988593
:103490000E944D0540E064EB8F8198850E941905DC
:1034A0008F8198850E94C604182F8F8198850E946D
:1034B0006C05111101C009831A818EA5803111F4A8
:1034C0000C949324BE01625D7F4FCE0101960E9451
:1034D0000406811790F48A818A838D818F5F8D83A2
:1034E0008EA5883231F0B0F4803119F0823209F0C3
:1034F000B1CF8E818F5F8E83ADCF8EA5803111F4D9
:103500008CE0EACFBE01625D7F4FCE0101960E9442
:103510000406E2CF8B3369F3823409F09BCFE9CF05
:103520008F8198850E946C0540E06CEC8F819885B6
:103530000E941905498164E48F8198850E941905CC
:103540008B81882379F1EA81E9506EEEC62E62E024
:10355000D62EE33038F4F0E0EE0FFF1FEA5EFE4FA8
:10356000C080D1808C81882309F461C08981811158
:103570005EC00E94A3044B015C010D2C000CEE0800
:10358000FF088F8198850E94C604813059F00E94FF
:10359000A3046C197D098E099F09681579058A05B0
:1035A0009B0578F38CE08A83F12CE12C0FE53FE753
:1035B000D32E4FE1C42E5FE3B52E8D818E151F04EF
:1035C00009F00CF499C04E2DBE01695C7F4FCE010D
:1035D00001960E94E10E1A811D3080F11CE08FA936
:1035E000803181F1BE01695C7F4FCE0101960E945E
:1035F0000406811709F478C0AE01425D5F4FBE0139
:10360000695C7F4FCE0101960E94A405882309F4CE
:103610006BC08FA9803109F467C01B3009F468C002
:103620001C3091F01A3009F065C0BAAA0EC0B6017C
:10363000DD0C880B990B0E949403B4CF193078F6F7
:1036400019E0CDCF8CE0D5CFDAAA8F8198850E9482
:103650006C05BE01695C7F4F8F8198850E944D0586
:1036600040E06EE48F8198850E94190540E068A9CA
:103670008F8198850E94190540E069A98F819885FE
:103680000E9419058FA9803131F040E06AA98F812D
:1036900098850E9419058F8198850E946C05BE014E
:1036A000695C7F4F8F8198850E944D05498168E450
:1036B0008F8198850E94190564E170E080E090E0B8
:1036C0000E9494038981882331F06AE070E080E0F1
:1036D00090E00E9494038F8198850E946C058A81F6
:1036E000811708F4812F8A833FEFE31AF30A65CF2D
:1036F0000AABABCFCAAAA9CF0E8110E00115110504
:1037000039F46BE575E082EB95E00E94B61118C1C3
:103710006DE571E082EB95E00E9480116801053053
:1037200011051CF024E0C22ED12C99E3A92E95E0BE
:10373000B92EF12CE12C4E2DBE01695C7F4FCE01DC
:1037400001960E94E10E81113EC020E030E04EEF74
:1037500052ECF50161917191819191915F010E940B
:1037600062322B013C01FFEFEF1AFF0A20E030E04C
:103770004CEF52EC0E94A93087FF71C0B701CE0117
:10378000C7960E948A116FE771E0CE018E960E9463
:10379000D611BE01695C7F4FCE018E960E94271123
:1037A00067ED71E00E9411116BE575E00E94271131
:1037B0000E94EA10CE018E960E948E10CE01C7960E
:1037C0000E948E1095C0AE01425D5F4FBE01695CE4
:1037D0007F4FCE0101960E94A405882309F4B5CF3E
:1037E0006FA570E0762F6627770F770F770F2EA5DE
:1037F00048E0249F90011124262B372B8FA980317C
:10380000D1F46DA970E08CA9DB01A81BB109CD0131
:103810009695982F8827979587950E947D35CB019F
:103820004097B901B3E0660F771FBA95E1F760786A
:103830009C01260F371F2138B4EE3B070CF485CFCF
:10384000B901330F880B990B0E94B03020E030E0B3
:1038500040E05CE30E940F319B01AC017ACF22E093
:10386000B301A201CE010330110509F454C1CF9672
:103870000E94A612B701CE01C7960E948A116FE777
:1038800071E0CE018E960E94D611BE01695C7F4F19
:10389000CE018E960E94271163E672E00E941111FC
:1038A000BE01615C7F4F0E942711BC0184E995E055
:1038B0000E94B611CE018E960E948E10CE01C79640
:1038C0000E948E10CE01CF960E948E1064E975E0A2
:1038D000CE018E960E94CD1160E472E0CE018E96EC
:1038E0000E9411110E94EA10CE018E960E948E1045
:1038F000EC14FD040CF41FCF82EB95E00E94CB0F7B
:1039000003301105A9F46AE072E0CE018E960E94A0
:10391000D61162EB75E0CE018E960E942711BC0194
:1039200082EB95E00E94B611CE018E960E948E1019
:1039300042E150E064E172E082EB95E00E94BE104B
:103940008091B6059091B705892B09F4C4C062EB4C
:1039500075E0CE0101960E94CD11CE0101960E9424
:103960003F12CE0101960E948E1062EB75E0CE01EF
:1039700080960E94CD1180912A03882309F4A7C064
:1039800080914F0390915003843191050CF09FC0BA
:103990000091040110910501013CF3E01F070CF0B8
:1039A00096C001969093500380934F030E94A30406
:1039B000C0902203D0902303E0902403F0902503CD
:1039C0006C197D098E099F090E94AE3020E030E01D
:1039D0004AE754E40E94CE32609326037093270393
:1039E0008093280390932903083C110534F488EC54
:1039F00090E09093050180930401809104019091DF
:103A000005012AE2C22E23E0D22E06E213E09C0139
:103A1000265233407901C701800F911F9A83898311
:103A2000D8016D918D01CE0101960E94DC12C01665
:103A3000D10689F7E0900401F0900501C7010496D2
:103A40009093050180930401BE01605E7F4FCE011B
:103A500001960E94CD11CE0101960E94F310BC0187
:103A600082EB95E00E94B611CE0101960E948E1065
:103A70004091B6055091B7054115510531F06BE203
:103A800073E082EB95E00E944E0F8FE4C82E83E036
:103A9000D82E0BE213E0F701E752F3407F01C70194
:103AA000800F911F9A838983D8016D918D01CE017A
:103AB00001960E94DC12C016D10689F7809104019C
:103AC0009091050184969093050180930401CE01A5
:103AD00080960E948E1064E670E080E090E00E9484
:103AE0009403C35BDF4F0FB6F894DEBF0FBECDBFAC
:103AF000DF91CF911F910F91FF90EF90DF90CF90CA
:103B0000BF90AF909F908F907F906F905F904F90FD
:103B10003F902F9008958E960E94A612BE01625D7E
:103B20007F4FCE01C7960E94CD1160E472E0CE01B6
:103B3000C7960E9411110E94EA10CE01C7960E94FA
:103B40008E10CE018E963CCE60E080E10E94230371
:103B50008091E9038111EBC02AE030E040E050E0C1
:103B60002E962CAF3DAF4EAF5FAF2E9767E272E05F
:103B700082EB95E00E948011312C212C28961FAEFB
:103B8000289729961FAE2997C12CD12C760102E3E4
:103B900010E0812C912C540180E10E945403092EE5
:103BA000000CAA0BBB0B880E991EAA1EBB1E65E05B
:103BB00070E080E090E00E9494030150110961F7E9
:103BC0004090350550903605609037057090380567
:103BD000C501B4010E94B03020E030E040EA50E47A
:103BE0000E940F3120E030E040E85AE30E940F319C
:103BF00020E030E048E452E40E94CE32A30192017A
:103C00000E94613220E030E040E751E40E940F3131
:103C10004B015C01A30192016AE979E989E390E42F
:103C20000E9461329B01AC01C501B4010E94CE32F9
:103C300020E030E0A9010E94623220E030E040E262
:103C400051E40E940F315B018C01232D322D289607
:103C50004FAD289729965FAD29970E94CA33181651
:103C600044F43A2C2B2C28960FAF289729961FAF97
:103C700029979FEFC91AD90AE90AF90A2E962CAD9D
:103C80003DAD4EAD5FAD2E972C153D054E055F0544
:103C90000CF07DCF6EE170E080E090E00E94940334
:103CA0006EE272E082EB95E00E94801122E0432DEB
:103CB000522D28966FAD289729967FAD2997CE0172
:103CC00001960E94A612BE016F5F7F4FCE018096C3
:103CD0000E94CD116BE372E0CE0180960E9411111B
:103CE000BC018AE995E00E94B611CE0180960E943F
:103CF0008E10CE0101960E948E1062E472E0CE0119
:103D000001960E94D6116AE975E0CE0101960E94E3
:103D1000271162EB75E00E942711BC0182EB95E050
:103D20000E94B611CE0101960E948E1009CE83E04A
:103D300090E0A0E0B0E02E968CAF9DAFAEAFBFAFED
:103D40002E9714CF68EC70E080E090E00E9494031E
:103D50000E94770A64E670E080E090E00E9494039D
:103D600062E370E080E090E00E94940349E050E05C
:103D70006CE171E086EE95E00E94820162E370E002
:103D800080E090E00E94940303E010E086EE95E06E
:103D90000E94A606892B61F149E050E06CE171E0D8
:103DA00086EE95E00E94820165E070E080E090E0A0
:103DB0000E949403F12CE12C86EE95E00E94A60669
:103DC00032E0E316F104A4F486EE95E00E94A60624
:103DD000892B39F086EE95E00E94BE064FEFE41A7B
:103DE000F40A65E070E080E090E00E949403E4CF84
:103DF00062E370E080E090E00E94940301501109BA
:103E000029F68AE090E00E947D0A6B017C0120E0A7
:103E100030E0A9010E94A930181634F08AE090E041
:103E20000E947D0A6B017C010BE010E020E030E095
:103E300042ED53E4C701B6010E94A930181684F080
:103E40000150110969F068EC70E080E090E00E9498
:103E5000940383E090E00E947D0A6B017C01E6CF31
:103E600020E030E0A901C701B6010E94A930181670
:103E70000CF047CC20E030E048EC52E4C701B6013A
:103E80000E94A93021E087FF20E0B701A601CE0102
:103E900001960E94A612BE016F5F7F4F82EB95E0F4
:103EA0000E944310CE0101960E948E1062EB75E0D5
:103EB000CE0101960E94CD1166E472E0CE0101961A
:103EC0000E941111BC0182EB95E00E94B611CE0157
:103ED00001960E948E106AE472E0CE0101960E9463
:103EE000D61162EB75E0CE01019615CF0E94A304B6
:103EF0004B015C0186EE95E00E94110764E670E0DC
:103F000080E090E00E9494030E94270764E670E03E
:103F100080E090E00E94940328961FAE2897D12C51
:103F2000C12C312C212C2A961FAE1EAE2A97FCEDF7
:103F30004F2EF5E05F2E612C712CCE0180962796D6
:103F40009FAF8EAF27970E94A304681979098A0949
:103F50009B09683B7B408105910508F06AC086EEAD
:103F600095E00E94A606892B09F450C04092EA050C
:103F70005092EB056092EC057092ED050E94DF0611
:103F800097FD44C082349105C9F78E010F5F1F4F22
:103F900078010E94DF0697FF40C089818D34B1F51A
:103FA000C8014D9630E020E0D8014D918D01240FDD
:103FB000311D8A179B07C1F72E5B3F4F8E8D90E016
:103FC000982F88274F8D840F911D28173907F1F4FA
:103FD0008C8190E0982F88272D81FC01E20FF11D44
:103FE0002A96FFAFEEAF2A972E80312C322C222456
:103FF0008F81280E311CC884D12CDC2CCC248985DF
:10400000C80ED11CF1E02896FFAF289762E370E05C
:1040100080E090E00E94940396CFF70181937F01A6
:1040200027962EAD3FAD27972E173F0709F0B1CF4A
:10403000B4CF0E94A304681979098A099B09683BD7
:104040007B4081059105A8F428963FAD289733233E
:1040500009F477C062E370E080E090E00E9494038E
:1040600086EE95E00E94110762E370E080E090E048
:104070007BC028964FAD2897442309F462C0B6014F
:10408000CE0180960E948A11B101CE018E960E94C7
:104090008A112A966EAD7FAD2A97CE01CF960E94E7
:1040A0008A11BE01615C7F4FCE01C7960E94CD117F
:1040B00060E472E0CE01C7960E941111BE01625DFC
:1040C0007F4F0E94271160E472E00E941111BE012F
:1040D000605E7F4F0E9427116FE472E00E94111111
:1040E000BC018AE995E00E94B611CE01C7960E94F4
:1040F0008E10CE01CF960E948E10CE018E960E9419
:104100008E10CE0180960E948E1065E572E082EBE3
:1041100095E00E94801162EB75E0CE0180960E94CE
:10412000CD116AE975E0CE0180960E942711BC018D
:1041300082EB95E00E94B611CE0180960E948E100F
:1041400089CF6BE575E082EB95E00E94B61182CFD6
:104150008091E903882321F082EB95E00E94AF0172
:1041600068EC70E080E090E00E949403E9CB10924C
:10417000E903E6CB81E08093E903809369058091B0
:10418000E3039091E4039093E2038093E103D8CB9F
:1041900064E670E080E090E00E9494038091080162
:1041A000909109010B9731F580911206882309F04F
:1041B000F89482E10E94C7038C0180911206882343
:1041C00009F078940115110509F4D5C080E090EC50
:1041D000A9E7B4EC8093050690930606A093070622
:1041E000B09308068093090690930A06A0930B06E5
:1041F000B0930C068091080190910901469731F522
:1042000080911206882309F0F89481E00E94C70388
:104210008C0180911206882309F07894011511050C
:1042200009F40AC180E090ECA9E7B4EC809305069C
:1042300090930606A0930706B0930806809309069C
:1042400090930A06A0930B06B0930C0664E670E008
:1042500080E090E00E949403012B09F071CBC090A4
:104260000906D0900A06E0900B06F0900C06C0926A
:104270001E03D0921F03E0922003F092210380914D
:10428000050690910606A0910706B0910806809356
:104290001A0390931B03A0931C03B0931D036DE5B9
:1042A00071E0CE0180960E94D61121E0B701A601EF
:1042B000CE0101960E94A612BE016F5F7F4FCE0114
:1042C00080960E944310CE0101960E948E1064EBEE
:1042D00071E0CE0101960E94D611BE01605E7F4F53
:1042E000CE0101960E94271165E672E00E9411112D
:1042F000BC0182EB95E00E94B611CE0101960E94AE
:104300008E1040911A0350911B0360911C03709111
:104310001D0321E0CE0101960E94A612BE016F5F2F
:104320007F4FCE0180960E944310CE0101960E94DD
:104330008E1069E672E0CE0101960E94D611BE0190
:10434000605E7F4FCE0101960E9427116CE672E0FD
:104350000E9411110E94EA10CE0101960E948E1057
:1043600064E670E080E090E00E949403CE018096C5
:104370000E948E10E5CA10910D06E0900E066E2D7B
:1043800070E090E080E00E94B0302DEC3CEC4CEC12
:104390005DE30E940F314B015C01612F70E090E002
:1043A00080E00E94B0309B01AC01C501B4010E94C5
:1043B0006232609305067093060680930706909319
:1043C000080600910F06F0901006602F6F7770E0DE
:1043D00090E080E00E94B0304B015C016F2D70E0F6
:1043E00090E080E00E94B0302DEC3CEC4CEC5DE3C2
:1043F0000E940F319B01AC01C501B4010E946232E1
:1044000007FD18C06093090670930A0680930B0697
:1044100090930C06812F8E0D800F8F0D01E010E020
:1044200090911106891302C010E000E011950195EA
:104430001109E0CE9058E6CF10910E0600910D06BE
:1044400060910D0670910E0676276727762790E01B
:1044500080E00E94AE302DEC3CEC4CEC5DE30E9421
:104460000F316093050670930606809307069093BC
:104470000806E0901006F0900F066F2D6F77762FEC
:104480006E2D90E080E00E94AE302DEC3CEC4CECC8
:104490005DE30E940F31F7FC18C06093090670932A
:1044A0000A0680930B0690930C06812F800F8E0DC9
:1044B0008F0D01E010E090911106891302C010E009
:1044C00000E0119501951109C1CE9058E6CF809179
:1044D0000701882309F434CA0E94630C2B013C01B4
:1044E0000E94D50B4B015C016091190570911A0572
:1044F00080911B0590911C050E94B03020E030E0B7
:1045000048EC52E40E94CE326B017C010E94630CA5
:1045100020E030E048EC52E40E94CE32A701960140
:104520000E94CE3221E03EED42E45EE30E94CF33B2
:104530006B017C0120E030E048EC52E4C301B201A1
:104540000E94CE32AB01BC0122E0CE0180960E94D7
:10455000A612BE01605E7F4FCE0101960E94CD1172
:104560006EE672E0CE0101960E941111BC0184E951
:1045700095E00E94B611CE0101960E948E10CE01E8
:1045800080960E948E1064E975E08AE995E00E94A9
:10459000B6116AEB71E0CE0101960E94D61164E972
:1045A00075E0CE0101960E942711BC0184E995E0D7
:1045B0000E94B611CE0101960E948E1021E0B50135
:1045C000A401CE0180960E94A612BE01605E7F4FBC
:1045D000CE0101960E94CD1163E772E0CE010196F3
:1045E0000E941111BC0182EB95E00E94B611CE0130
:1045F00001960E948E10CE0180960E948E1064EB70
:1046000071E0CE0101960E94D61162EB75E0CE01F9
:1046100001960E94271166E772E00E941111BC0109
:1046200082EB95E00E94B611CE0101960E948E1099
:10463000A701960160E070E080E89FE30E9461328C
:1046400020E03AE24DE257E40E940F31AB01BC0199
:1046500021E0CE0180960E94A612BE01605E7F4FCF
:10466000CE0101960E94CD1168E472E0CE01019660
:104670000E9411110E94EA10CE0101960E948E1034
:10468000CE0180960E948E1064E975E0CE010196FD
:104690000E94CD1162EB75E0CE0101960E942711B8
:1046A000BC0182EB95E00E94B611CE0101960E94FA
:1046B0008E1065E070E080E090E056CD3BE0E32EA8
:1046C000F12C10E000E09924939443E2842E909220
:1046D000400480926204109241041092630462E0EC
:1046E00083E20E9420091092F3038093F20381E099
:1046F00095E00E94FE09D82EC12C81E095E00E9431
:10470000FE095C01AC28BD280E943908B50190E083
:1047100080E00E94AE302AE939E949E95FE30E946E
:10472000CE320E9447330617170708F48B0162E365
:1047300070E080E090E00E94940351E0E51AF108F7
:1047400031F66AE772E082EB95E00E94801119A2CF
:1047500018A21BA21AA21DA21CA24AE0BE016F5FF2
:104760007F4FC8010E94D72CBE016F5F7F4FCE01E3
:1047700080960E948011BE01605E7F4FCE0101963F
:104780000E94CD116AE872E0CE0101960E941111DB
:10479000BC018AE995E00E94B611CE0101960E9403
:1047A0008E10CE0180960E948E106FE872E0CE01CE
:1047B00001960E94D6116AE975E0CE0101960E9429
:1047C000271162EB75E00E942711BC0182EB95E096
:1047D0000E94B611CE0101960E948E1045CC81E058
:1047E000809306010E944A048C0162E972E082EB28
:1047F00095E00E94801160E074E0601B710BCE01B7
:1048000001960E948A11CE0101960E94EA10CE0103
:104810000196AECD62EA72E082EB95E00E948011D3
:104820000E944A04BC01EBCFF0E0E0E0099588C8A3
:104830008091630518160CF055C081E080936105E6
:104840006DEA72E082EB95E00E9480118091610533
:10485000882309F44AC06BEB72E0CE0101960E94F6
:10486000D61162EB75E0CE0101960E942711BC01C2
:1048700082EB95E00E94B611CE0101960E948E1047
:1048800062EB75E0CE0101960E94CD11CE0101963A
:104890000E943F12CE0101960E948E1068EE73E0D6
:1048A00080E090E00E9494038091610581110E9454
:1048B00099246DE571E082EB95E00E948011809172
:1048C000E9038093690581113BC861ED71E086EAD7
:1048D00095E00E94801186EE9FEF9093E403809311
:1048E000E3032EC810926105ABCF63EC72E0CE01FA
:1048F00001960E94D61162EB75E0CE0101960E94EE
:104900002711BC0182EB95E00E94B611CE01019601
:104910000E948E10D4CF6CEC72E082EB95E00E9486
:1049200080110C94A01C1D3010F00C946B1A0C9488
:10493000801A0F931F93CF93DF9301E615E0D0E029
:10494000C0E00A5F1F4F80916305082E000C990B91
:10495000C817D9076CF4F801878190850E949A19CD
:1049600068EE73E080E090E00E9494032196E9CF26
:10497000DF91CF911F910F9108951F920F920FB663
:104980000F9211242F933F934F935F936F937F93D5
:104990008F939F93AF93BF93EF93FF9384E694E03D
:1049A0000E941902FF91EF91BF91AF919F918F915A
:1049B0007F916F915F914F913F912F910F900FBE1B
:1049C0000F901F9018951F920F920FB60F921124FF
:1049D0002F938F939F93EF93FF93E0917404F09143
:1049E00075048081E0917A04F0917B0482FD1BC004
:1049F000908180917D048F5F8F7320917E04821758
:104A000041F0E0917D04F0E0EC59FB4F958F8093ED
:104A10007D04FF91EF919F918F912F910F900FBE89
:104A20000F901F9018958081F4CF1F920F920FB6B0
:104A30000F9211242F933F938F939F93AF93BF9324
:104A40008091D6039091D703A091D803B091D90358
:104A50003091D50323E0230F2D3758F50196A11D82
:104A6000B11D2093D5038093D6039093D703A093D1
:104A7000D803B093D9038091DA039091DB03A0911E
:104A8000DC03B091DD030196A11DB11D8093DA0313
:104A90009093DB03A093DC03B093DD03BF91AF9150
:104AA0009F918F913F912F910F900FBE0F901F906C
:104AB000189526E8230F0296A11DB11DD2CF1F9293
:104AC0000F920FB60F9211242F933F934F935F9342
:104AD0006F937F938F939F93AF93BF93EF93FF93C6
:104AE000E091F003F091F103309749F0A685B78586
:104AF0008585968D91FF14C09C918923A1F4FF9127
:104B0000EF91BF91AF919F918F917F916F915F9145
:104B10004F913F912F910F900FBE0F901F901895BE
:104B20009C91892361F7A389B4899C91858980959B
:104B300089238C93868997890197F1F7608D718D10
:104B4000A685B785558538E020E0CB010197F1F7C0
:104B5000822F90E095958795282F4C91452309F059
:104B60002068315091F7868D81FD20958091EF036B
:104B700090E001968F7399273091EE03381799F0E2
:104B8000A091EF03B0E0AB56BC4F2C938093EF03A2
:104B9000828D938D0197F1F7A389B4898C919589C2
:104BA000892B8C93ACCF868D8160868FF1CF1F923D
:104BB0000F920FB60F9211242F933F934F935F9351
:104BC0006F937F938F939F93AF93BF93EF93FF93D5
:104BD0008091B900887F803609F44AC0F0F58832A8
:104BE00009F4A7C018F5803109F49BC0B8F48823F4
:104BF00009F4F9C0883009F494C0FF91EF91BF9196
:104C0000AF919F918F917F916F915F914F913F9164
:104C10002F910F900FBE0F901F901895883109F4B7
:104C200088C0803251F78093380414C0803409F46E
:104C30009DC040F48033B9F38833F9F6809338048B
:104C400085ECB0C0803509F485C0883509F496C07C
:104C5000883499F60E94880FD0CF883909F48CC027
:104C600038F5883729F050F4883611F0803729F666
:104C700083E080933A041092940357C0883809F473
:104C80007BC0803919F0803809F0B7CF8091940348
:104C9000803208F071C0E091940381E08E0F809320
:104CA00094038091BB00F0E0EC58FC4F80833DC042
:104CB000803B39F0E0F4803A09F479C0883A09F091
:104CC0009CCF84E080933A04109273031092720395
:104CD000E091EC03F091ED0309958091720381114D
:104CE0000FC081E0809372031092520309C0803C90
:104CF00009F4A6CF883C09F4A3CF883B09F07DCF07
:104D0000E091730381E08E0F80937303F0E0EE5A1D
:104D1000FC4F80818093BB0090917303809172035C
:104D200029C0809115048093BB0085EC8093BC0062
:104D300064CF9091370480913604981758F5E0912C
:104D4000370481E08E0F80933704F0E0EA5EFB4F7A
:104D50008081E9CFE091370481E08E0F80933704A2
:104D60008091BB00F0E0EA5EFB4F808390913704B6
:104D7000809136049817C8F285E8D8CFE0913704BF
:104D800081E08E0F809337048091BB00F0E0EA5EF3
:104D9000FB4F80838091390481115CCF81E0809347
:104DA000140484EA8093BC0010923A0426CF85EC68
:104DB0008093BC0010923A0480919403803230F4C6
:104DC000E0919403F0E0EC58FC4F10826091940362
:104DD00070E0E091EA03F091EB0384E793E009953A
:104DE000109294030ACF1092380434CF10926704C3
:104DF0001092660488EE93E0A0E0B0E0809368042F
:104E000090936904A0936A04B0936B0429E231E0A3
:104E1000309365042093640425EC30E030937104F2
:104E20002093700424EC30E03093730420937204D8
:104E300020EC30E0309375042093740421EC30E0D2
:104E4000309377042093760422EC30E03093790499
:104E50002093780426EC30E030937B0420937A048E
:104E600010927D0410927E0410927F0410928004B0
:104E70001092040510920305809305059093060592
:104E8000A0930705B09308052BE331E030930205AA
:104E900020930105109212061092E9051092E80580
:104EA0008093EA059093EB05A093EC05B093ED0594
:104EB0008DE491E09093E7058093E6051092FD055F
:104EC0001092FC051092FF051092FE05109201064B
:104ED00010920006109203061092020660910406DA
:104EE0006E7F6D7F609304066695617081E0682730
:104EF00089E00E94F50261E089E00E942303EAE96B
:104F0000F2E0E491E093F605E6E8F2E0E491F0E007
:104F1000EE0FFF1FED58FD4F859194919093F8058A
:104F20008093F70560E08AE00E94230380910406E5
:104F300081FD04C061E08AE00E94F5028AE080936E
:104F4000F205EBE9F2E0E491E093F305E7E8F2E043
:104F5000E491F0E0EE0FFF1FE759FD4F859194912A
:104F60009093F5058093F4058FEF8093C1058093AE
:104F7000C2058093C3058093C4056DE571E082EBA3
:104F800095E00E94D6116DE571E08CEA95E00E94F3
:104F9000D6116DE571E086EA95E00E94D6116DE5C7
:104FA00071E080EA95E00E94D6116DE571E08AE932
:104FB00095E00E94D6116DE571E084E995E00E94CC
:104FC000D6116AED72E08EE895E00E94D61161EE8E
:104FD00072E088E895E00E94D6111092610585E0A4
:104FE0008093620510926305109265051092640526
:104FF0001092670510926605109268051092690577
:1050000066EE72E08BE595E00E94D61186E190E0B5
:1050100090930E0580930D058CE79CE8A1E0B0E02D
:105020008093190590931A05A0931B05B0931C0556
:1050300081EA97E6A3E3BDEB80931D0590931E05DF
:10504000A0931F05B093200586E696E6A6EABFE387
:105050008093210590932205A0932305B093240506
:1050600081E080932D0529E130E030932F052093D6
:105070002E058093300580E090E4ACE1B5E48093A8
:10508000310590933205A0933305B0933405109207
:105090003505109236051092370510923805E9E370
:1050A000F5E080E1DF011D928A95E9F7109249054C
:1050B00010924A0510924B0510924C0510924D0526
:1050C00010924E0510924F05109250051092510506
:1050D00010925205109253051092540510925505E6
:1050E00010925605109257051092580581E090E0F5
:1050F00090935A05809359050895CF93DF93CDB7C8
:10510000DEB72C970FB6F894DEBF0FBECDBF7894F4
:1051100084B5826084BD84B5816084BD85B58260BC
:1051200085BD85B5816085BD80916E00816080936D
:105130006E001092810080918100826080938100D6
:1051400080918100816080938100809180008160E6
:10515000809380008091B10084608093B100809141
:10516000B00081608093B00080917A008460809369
:105170007A0080917A00826080937A0080917A0030
:10518000816080937A0080917A00806880937A00B1
:105190001092C10061E08EE00E942303E09174044C
:1051A000F091750482E08083E0917004F0917104C5
:1051B0001082E0917204F09173048FEC808310925E
:1051C0007C04E0917804F091790486E08083E0919A
:1051D0007604F0917704808180618083E091760489
:1051E000F0917704808188608083E0917604F0916B
:1051F0007704808180688083E0917604F091770461
:1052000080818F7D808360E08EE00E94F5020E94A5
:10521000010881E08093400483E28093620410924D
:1052200041041092630460E181E095E00E94450A28
:105230000E9439088FE39CE90197F1F700C0000054
:1052400068EC70E080E090E00E94940384E690E0D7
:1052500090930B0180930A010E94D0318093DE036A
:1052600085E690E00E94D0318093DF030091DE0359
:105270001091DF03B801012E000C880B990B0E94DE
:10528000B0309B01AC010E941F34811106C00B504D
:1052900011090C30110508F4ECC084E690E00E947E
:1052A000F51231E6C32E35E0D32E56010EE110E0A3
:1052B000C8010E94D031F50181935F010F5F1F4F3C
:1052C00007321105A9F710916205612F012E000C1C
:1052D000770B880B990B0E94B0309B01AC010E94A8
:1052E0001F34811103C0153009F4EEC08EE190E047
:1052F0000E941E1368EC70E080E090E00E9494032E
:1053000062EF72E082EB95E00E9480110E9401083A
:1053100064E670E080E090E00E9494036EE875E03F
:10532000CE0101960E94CD11CE0101960E94F3108C
:105330000E94EA10CE0101960E948E1062EB75E089
:10534000CE0101960E94CD11CE0101960E943F121E
:10535000CE0101960E948E1086E78093B805809159
:10536000C1058F3F11F40E9401088091C1058F3F54
:1053700001F58091B80591E0909340048093620418
:10538000109241041092630460ED81E095E00E9468
:10539000450A0E94390861E08091B8050E94200901
:1053A0001092F3038093F20381E095E00E94FE09DE
:1053B000F82EF8E5FF1609F495C06BEF72E082EB6A
:1053C00095E00E9480111092070162EB75E0CE011A
:1053D00001960E94CD11CE0101960E943F12CE018E
:1053E00001960E948E108AE2C82ED12C98EE892E4A
:1053F00093E0992EA12CB12C20E0E22E20E0F22E99
:1054000001E06DE571E0CE0107960E94D61110E033
:1054100084E694E00E94F901181619060CF0D3C036
:105420001111D1C084E694E00E94D7018A3009F0BE
:105430007AC11091E003112309F48AC18091A40577
:105440009091A505892B09F47CC167E073E0CE013A
:1054500001960E94D611BE01695F7F4FCE01019671
:105460000E9427110E94AF01CE0101960E948E106A
:1054700068C14DE0C42E45E0D42E04E610E0C8011A
:105480000E94D031F60181936F010F5F1F4F023BE5
:105490001105A9F780910D0590910E0590930901D2
:1054A000809308016FE075E0CE0101960E94D6114D
:1054B000BE016F5F7F4F8EE895E00E944310CE01E2
:1054C00001960E948E10EDCE0EE110E0C8010E9400
:1054D000D031F60181936F010F5F1F4F0534110525
:1054E000A9F708CF88E80E941D0F9093C605809306
:1054F000C5058AE80E941D0F9093C8058093C705D3
:105500008CE80E941D0F9093CA058093C9058EE810
:105510000E941D0F9093CC058093CB0580E90E94DB
:105520001D0F9093CE058093CD0582E90E941D0F3B
:105530009093D0058093CF0584E90E941D0F90932E
:10554000D2058093D10586E90E941D0F9093D40562
:105550008093D30588E90E941D0F9093D605809310
:10556000D5058AE90E941D0F9093D8058093D70531
:105570008CE90E941D0F9093DA058093D9058EE97E
:105580000E941D0F9093DC058093DB058091C1057F
:105590008F3F09F028CF8091B80591E090934004A7
:1055A00080936204109241041092630464EF81E0DE
:1055B00095E00E94450A6FE381E095E00E94450A6C
:1055C0000E94390810CF8B859C85892B51F084E689
:1055D00094E00E94880264E170E080E090E00E9424
:1055E0009403BE01695F7F4F80EA95E00E944310FB
:1055F000CE0107960E948E106DE571E082EB95E07A
:105600000E9480118091A4059091A505813091059B
:1056100009F0C6C060EA75E08CEA95E00E94B61118
:105620000E94710F6CEA75E0CE0101960E94CD11C7
:105630008D819E81892B09F4A5C0E981FA8130977B
:1056400009F4A0C08081823409F484C0833409F451
:105650008EC0813409F096C060E173E080EA95E085
:105660000E948011CE0101960E948E1080EA95E082
:105670000E94C00FCB010E949A198091E9038823F0
:1056800009F43FC00E94A304A50194010E94303296
:10569000CA01B9010E94AE302091E5033091E603C2
:1056A0004091E7035091E8030E94613220910C0180
:1056B00030910D0140910E0150910F010E94CA33AB
:1056C0001816FCF48091E3039091E4034A9609F4E0
:1056D000BFC08091E1039091E2030E949A190E9459
:1056E000A304A50194010E943032CA01B9010E94AD
:1056F000AE306093E5037093E6038093E7039093E5
:10570000E8036AE070E080E090E00E949403E11416
:10571000F10409F476CE0E940502882309F471CEC3
:105720000E9400006ECE8D3009F483CE89831A82E8
:1057300041E050E0BE016F5F7F4FCE0107960E94AF
:10574000BE106AE070E080E090E00E94940360CEBA
:1057500011E0F7CF63E173E080EA95E00E948011E9
:105760001092E9038CEF9FEF0E949A197BCF66E1BC
:1057700073E080EA95E00E9480110093E9038DEFC9
:105780009FEFF2CFBE016F5F7F4F80EA95E00E94EE
:10579000B6116AE070E080E090E00E94940362CF6E
:1057A000049768F562ED71E0CE0101960E94D61172
:1057B000BE016F5F7F4F80EA95E00E942810182F8E
:1057C000CE0101960E948E101123C9F08091A4058C
:1057D0009091A505029788F0E091A005F091A105B0
:1057E000309759F0818180330CF4845E9601281B38
:1057F000310987FD3395C9013ECF80E0F6CF60EADD
:1058000075E08CEA95E00E94B6110E94710F1A8231
:1058100019821C821B821E821D8261E572E0CE010C
:1058200001960E943A11BE016F5F7F4F8CEA95E0AE
:105830000E942810182FCE0101960E948E1011236D
:1058400021F0F0E0E0E0099518CF0E94471315CF52
:1058500080916105882309F442CF0E9499243FCFAB
:105860008BE595E00E948E1088E895E00E948E10EE
:105870008EE895E00E948E1084E995E00E948E10DB
:105880008AE995E00E948E1080EA95E00E948E10D1
:1058900086EA95E00E948E108CEA95E00E948E10B8
:1058A00082EB95E00E948E108DE491E09093E705E5
:1058B0008093E60586EE95E00C941107EF920F9326
:1058C0001F93CF93DF93E80134E047FD34E1042ECA
:1058D000000C550B57FF03C0519541955109E32E1C
:1058E000022F242FAE010E94F12CCE01DF91CF9127
:1058F0001F910F91EF900895662777270C94502EF3
:105900001F93FC0199278827BC01E894119110325C
:10591000E9F3193010F01E30C8F31B3251F01D327C
:1059200049F4689406C00E94C22C610F711D811D4C
:10593000911D119110531A30B0F33EF4909580955B
:10594000709561957F4F8F4F9F4F1F910895FB0179
:10595000DC0105900D920020E1F70895FC0105900F
:105960000020E9F7809590958E0F9F1F0895BB2723
:105970004A3031F4992322F4BDE2909581959F4FEE
:105980000C94D82C592F482F372F262F660F771FAE
:10599000881F991F660F771F881F991F620F731F3B
:1059A000841F951F660F771F881F991F0895BB27B7
:1059B000FB015527AA27880F991FAA1FA41710F0CB
:1059C000A41B83955051B9F7A05DAA3308F0A95DD7
:1059D000A193009779F7B111B1931192CB010C9477
:1059E0009930A9E0B0E0E7EFFCE20C94FF316A01E6
:1059F000F22EB02E102FFBE3AF2EA01608F41BE3FF
:105A00001F5F012F27E0AE014F5F5F4F0E94A02F65
:105A1000BC018981982F9970913009F43FC09BE2B5
:105A2000E1FC04C09E2D9170E0FC3AC05E2D5071E7
:105A3000E82FE87083FF46C084E0911101C083E045
:105A4000EF2DE81B8F1508F0E0E0D6018E2F20E245
:105A5000552351F1992329F0D6019C93C601019653
:105A60006C0196012D5F3F4FE2FE24C08EE4D6010B
:105A70008C9391E411969C93119712968C93D90173
:105A80008E2F90E281111BC0E20FF32FF11D1082C7
:105A90008EEF9FEF2996ECE00C941B329DE2C6CF6F
:105AA00090E2C4CF2D9381508111FCCFCE0ED11C3A
:105AB000E0E0D0CF8EE6D6018C9391E6DBCF9D93CC
:105AC0008150E0CF482F447082FF3DC084E09111A7
:105AD00001C083E08F1510F4EF2DE81BD6018E2F47
:105AE00020E2552309F1992329F0D6019C93C601A0
:105AF00001966C0196012D5F3F4FE2FE1BC089E4C9
:105B0000D6018C938EE411968C93119786E41296AD
:105B10008C93D9018E2F90E2882309F4B5CF9D9301
:105B20008150FACF2D9381508111FCCFCE0ED11C24
:105B3000E0E0D9CF89E6D6018C938EE611968C935E
:105B4000119786E6E4CF9B0177FF02C030E020E0AA
:105B5000A1E0B0E0911102C0B0E0A0E0F9013196FF
:105B6000AE0FBF1F8B2C912CBB2009F461C05401D8
:105B7000EFEFAE1ABE0AAA0DBB1DFA161B0619F0EE
:105B800014F04F2D4A1B511188C0E3FC59C0760117
:105B9000A42FB0E2A1114FC0C40ED11C992309F467
:105BA0005BC040E0D6011196F60190836D0155234C
:105BB00009F448C0012F060F9A81582F507184FFB5
:105BC00003C0913309F4015010160CF047C009309E
:105BD00008F008E0EEE2FE2E5B01A01AB108850194
:105BE0009194819491082F3F320729F4D601FC92B9
:105BF000F60131966F016217730794F102171307CC
:105C00007CF5DB01A21BB30BAA24A394B12CAC0E30
:105C1000BD1EAA0DBB1D11968C9121503109D601D4
:105C2000119628153905F4F0F60180836D01DBCF5C
:105C3000B12CA12CA0CFF701B1937F01A150AACF25
:105C40009111B0CFD601942F50E302C05D939150D3
:105C50009111FCCFC40ED11C40E0ACCF01E0BACF13
:105C600080E3DBCF6217730731F4963388F4953302
:105C700011F4552369F0F6018083FD01842F90E231
:105C8000811108C0A40FB11D1C9290E080E002CFEA
:105C900081E3F1CF91938150F3CF911183CF8ACFDC
:105CA000B0E0A0E0E6E5FEE20C94FF315C017B0190
:105CB0006115710519F0DB018D939C9385010F5FD0
:105CC0001F4FF501D0818D2F90E00E9478306C013C
:105CD000892BB9F5DD32B9F50F5F1F4FD50111964C
:105CE000DC91C1E05801F1E0AF1AB10843E050E0A7
:105CF00062EF70E0C5010E948130892B69F568016F
:105D000082E0C80ED11C45E050E06DEE70E0C601A7
:105D10000E948130892B21F4680197E0C90ED11CC3
:105D2000E114F10419F0D701CD92DC9260E070E04B
:105D300080E89FEFC111FFC060E070E080E89FE75E
:105D4000FAC05801BBCFDB3229F485010E5F1F4F2B
:105D5000F501D181C0E0C6CF43E050E06AEE70E0CB
:105D6000C5010E948130892BE9F0F80110E000E0C4
:105D700020E030E0A9015F01B0ED8B2E8D0E89E0AF
:105D80008815C8F19C2E689491F88C2F8870C2FFFA
:105D900016C0811102C00F5F1F4F3196D501DC91F3
:105DA000C92DE9CFE114F10429F00E5F1F4FF7016F
:105DB0001183008360E070E080EC9FE7BCC0882323
:105DC00011F001501109A5E0B0E00E94E6319B01FD
:105DD000AC01220F331F441F551F280D311D411DDB
:105DE000511D283999E93907490799E15907A8F25E
:105DF000C6609C2ED2CFAEEF8A1206C0C3FD3CC057
:105E00009C2E689493F8C9CFDF7DD534A9F58081A5
:105E10008D3239F4C061DF011296818162E070E059
:105E200006C0DF018B32C1F3119661E070E0805350
:105E30005D01A61AB70A8A30F8F4E0E8CE16ECE065
:105E4000DE065CF4B601660F771F660F771FC60E7D
:105E5000D71ECC0CDD1CC80ED11C5D01FFEFAF1AA4
:105E6000BF0A8C9180538A30A8F1C4FF03C0D1943B
:105E7000C194D1080C0D1D1DC1FF09C0E114F1042E
:105E800031F081E0A81AB108D701AD92BC92CA01E5
:105E9000B9010E94AE30C370C33009F490584B0171
:105EA0005C0120E030E0A9010E94A930882309F4B8
:105EB00040C0C1E2D1E017FF05C01195019511095D
:105EC000C9E0D1E06E01B8E1CB1AD10880E2E82E3A
:105ED000F12C0FC0D501B1CFFE012591359145912F
:105EE00054910E191F09C501B4010E940F314B01D5
:105EF0005C01D501C4010E151F0574F72497F594B4
:105F0000E794CC16DD06A9F78A2F880F8B2F881F00
:105F10008F3F49F020E030E0A901C501B4010E94A3
:105F2000A930811106C082E290E09093140680931C
:105F30001306C501B401CDB7DEB7ECE00C941B32FB
:105F4000283008F027E03327DA01990F311D87FD4B
:105F5000916000966105710539F432602E5F3D93C2
:105F600030E32A95E1F708959F3F30F080387105BE
:105F7000610509F03C5F3C5F3D93913008F080681B
:105F8000911DDF93CF931F930F93FF92EF92192FE1
:105F9000987F9695E92F96959695E90FFF27E158FA
:105FA000FE4F99273327EE24FF24A701E701059030
:105FB0000894079428F4360FE71EF81E491F511D58
:105FC000660F771F881F991F0694A1F70590079405
:105FD00028F4E70EF81E491F561FC11D770F881FB2
:105FE000991F661F0694A1F70590079428F4F80EF0
:105FF000491F561FC71FD11D880F991F661F771F86
:106000000694A1F70590079420F4490F561FC71F67
:10601000D81F990F661F771F881F0694A9F78491D0
:106020001095177041F0D695C79557954795F794F9
:10603000E7941A95C1F7E5E2F1E06894159015919F
:1060400035916591959105907FE27395E118F10A7C
:10605000430B560BC90BD009C0F7E10CF11E431FCF
:10606000561FC91FD01D7EF4703311F48A95E6CFF8
:10607000E894015030F0080F0AF40027021708F4E2
:10608000202F2395022F7A3328F079E37D932A95E8
:10609000E9F710C07D932A9589F606949795679540
:1060A000379517951794E118F10A430B560BC90B56
:1060B000D00998F023957E9173957A3308F070E3B8
:1060C0007C932013B8F77E9170617D9330F08395B7
:1060D00071E37D9370E32A95E1F71124EF90FF902F
:1060E0000F911F91CF91DF91992787FD909508958A
:1060F00091110C947C31803219F089508550C8F789
:106100000895FB01DC014150504088F08D918134AD
:106110001CF08B350CF4805E659161341CF06B359E
:106120000CF4605E861B611171F3990B0895881B56
:10613000FCCFDC01FC01672F71917723E1F73297E7
:1061400004C07C916D9370836291AE17BF07C8F352
:1061500008950E94EB3008F481E00895E89409C0A6
:1061600097FB3EF490958095709561957F4F8F4F8A
:106170009F4F9923A9F0F92F96E9BB279395F695A0
:10618000879577956795B795F111F8CFFAF4BB0F1E
:1061900011F460FF1BC06F5F7F4F8F4F9F4F16C082
:1061A000882311F096E911C0772321F09EE8872F0C
:1061B000762F05C0662371F096E8862F70E060E0C8
:1061C0002AF09A95660F771F881FDAF7880F969541
:1061D000879597F90895990F0008550FAA0BE0E8E5
:1061E000FEEF16161706E807F907C0F01216130699
:1061F000E407F50798F0621B730B840B950B39F4D9
:106200000A2661F0232B242B252B21F408950A263E
:1062100009F4A140A6958FEF811D811D08950E946C
:1062200022310C9496310E94883138F00E948F31CF
:1062300020F0952311F00C947F310C9485311124BA
:106240000C94CA310E94A73170F3959FC1F3950F4A
:1062500050E0551F629FF001729FBB27F00DB11DEA
:10626000639FAA27F00DB11DAA1F649F6627B00D7A
:10627000A11D661F829F2227B00DA11D621F739F63
:10628000B00DA11D621F839FA00D611D221F749F71
:106290003327A00D611D231F849F600D211D822FB8
:1062A000762F6A2F11249F5750409AF0F1F08823DF
:1062B0004AF0EE0FFF1FBB1F661F771F881F91500C
:1062C0005040A9F79E3F510580F00C947F310C940B
:1062D000CA315F3FE4F3983ED4F38695779567958E
:1062E000B795F795E7959F5FC1F7FE2B880F911D36
:1062F0009695879597F9089599278827089597F98E
:106300009F6780E870E060E008959FEF80EC08955B
:1063100000240A9416161706180609060895002484
:106320000A9412161306140605060895092E0394FE
:10633000000C11F4882352F0BB0F40F4BF2B11F472
:1063400060FF04C06F5F7F4F8F4F9F4F089557FDD1
:106350009058440F551F59F05F3F71F04795880FD3
:1063600097FB991F61F09F3F79F08795089512166A
:1063700013061406551FF2CF4695F1DF08C0161616
:1063800017061806991FF1CF8695710561050894C7
:106390000895E894BB2766277727CB0197F90895DE
:1063A000F999FECF92BD81BDF89A992780B50895DD
:1063B000262FF999FECF1FBA92BD81BD20BD0FB621
:1063C000F894FA9AF99A0FBE019608950E945232F3
:1063D000A59F900DB49F900DA49F800D911D112439
:1063E0000895B7FF0C94E6310E94E631821B930BAF
:1063F00008952F923F924F925F926F927F928F9269
:106400009F92AF92BF92CF92DF92EF92FF920F9343
:106410001F93CF93DF93CDB7DEB7CA1BDB0B0FB64D
:10642000F894DEBF0FBECDBF09942A88398848880A
:106430005F846E847D848C849B84AA84B984C884A0
:10644000DF80EE80FD800C811B81AA81B981CE0F97
:10645000D11D0FB6F894DEBF0FBECDBFED0108957C
:10646000A1E21A2EAA1BBB1BFD010DC0AA1FBB1F58
:10647000EE1FFF1FA217B307E407F50720F0A21BCA
:10648000B30BE40BF50B661F771F881F991F1A9437
:1064900069F760957095809590959B01AC01BD0161
:1064A000CF010895A29FB001B39FC001A39F700DBB
:1064B000811D1124911DB29F700D811D1124911D0C
:1064C00008955058BB27AA270E9479320C94963120
:1064D0000E94883138F00E948F3120F039F49F3FBC
:1064E00019F426F40C9485310EF4E095E7FB0C9436
:1064F0007F31E92F0E94A73158F3BA17620773075B
:106500008407950720F079F4A6F50C94C9310EF4B0
:10651000E0950B2EBA2FA02D0B01B90190010C01B3
:10652000CA01A0011124FF27591B99F0593F50F4CB
:10653000503E68F11A16F040A22F232F342F442723
:10654000585FF3CF469537952795A795F04053951B
:10655000C9F77EF41F16BA0B620B730B840BBAF0EB
:106560009150A1F0FF0FBB1F661F771F881FC2F756
:106570000EC0BA0F621F731F841F48F4879577956A
:106580006795B795F7959E3F08F0B0CF9395880F24
:1065900008F09927EE0F9795879508950E94E232AB
:1065A0000C9496310E948F3158F00E94883140F04F
:1065B00029F45F3F29F00C947F3151110C94CA31BA
:1065C0000C9485310E94A73168F39923B1F35523C8
:1065D00091F3951B550BBB27AA27621773078407F6
:1065E00038F09F5F5F4F220F331F441FAA1FA9F38C
:1065F00035D00E2E3AF0E0E832D091505040E6957A
:10660000001CCAF72BD0FE2F29D0660F771F881FDA
:10661000BB1F261737074807AB07B0E809F0BB0BCD
:10662000802DBF01FF2793585F4F3AF09E3F5105E1
:1066300078F00C947F310C94CA315F3FE4F3983EBC
:10664000D4F3869577956795B795F7959F5FC9F7CA
:10665000880F911D9695879597F90895E1E0660F4B
:10666000771F881FBB1F621773078407BA0720F0C4
:10667000621B730B840BBA0BEE1F88F7E09508952D
:106680000E9447336894B1110C94CA3108950E9456
:10669000AF3188F09F5798F0B92F9927B751B0F0D4
:1066A000E1F0660F771F881F991F1AF0BA95C9F796
:1066B00014C0B13091F00E94C931B1E008950C943A
:1066C000C931672F782F8827B85F39F0B93FCCF3ED
:1066D000869577956795B395D9F73EF49095809513
:1066E000709561957F4F8F4F9F4F089597FB16F4DC
:1066F0000E94BA330C947D33E894F92F96EBFF2374
:1067000081F0121613061406440B9395F69587959F
:106710007795679557954040FF23B9F71BC0992798
:106720000895882351F49850D2F7872B762F652F40
:10673000542F432F322F20E0B1F312161306140604
:10674000440B88233AF09A95440F551F661F771F14
:10675000881FCAF755234AF4440F551F11F460FFF0
:1067600004C06F5F7F4F8F4F9F4F880F969587951F
:1067700097F90895909580957095609550954095FE
:10678000309521953F4F4F4F5F4F6F4F7F4F8F4F4A
:106790009F4F08950E94EB3008F48FEF0895FA019F
:1067A000EE0FFF1F309621053105A1F1611571052E
:1067B00061F48038BFE39B0749F168949038810504
:1067C00061F08038BFEF9B0741F099234AF5FF3F06
:1067D000E1053105210519F1E8940894E795D901FF
:1067E000AA2329F4AB2FBE2FF85FD0F310C0FF5FB0
:1067F00070F4A695E0F7F73950F019F0FF3A38F445
:106800009F779F930DD00F9007FC9058089546F006
:106810000C94853160E070E080E89FE308954FE7D5
:106820009F775F934F933F932F930E94CF342F9185
:106830003F914F915F910E940F310C942C340E9434
:10684000EB30880B990B089529F416F00C947F31E6
:106850000C94C9310C9485310E94AF31A8F396385D
:10686000A0F707F80F92E8942BE33AEA48EB5FE7CA
:106870000E9425310F920F920F924DB75EB70F9283
:106880000E941735E8E6F0E00E945E344F915F9178
:10689000EF91FF91E595EE1FFF1F49F0FE57E0686D
:1068A0004427EE0F441FFA95E1F74195550B0E94DE
:1068B00091340F9007FE0C9485340895DF93CF93A5
:1068C0001F930F93FF92EF92DF927B018C016894EC
:1068D00006C0DA2EEF010E942231FE01E894A59154
:1068E0002591359145915591A6F3EF010E9479329A
:1068F000FE019701A801DA9469F7DF90EF90FF900D
:106900000F911F91CF91DF9108959B01AC0160E041
:1069100070E080E89FE30C94CE320C947F310C94AD
:106920004B350E94AF31D8F39923C9F3940F511D11
:10693000A3F39150504094F059F0882332F0660F41
:10694000771F881F91505040C1F79E3F51052CF78B
:10695000880F911D9695879597F908955F3FACF044
:10696000983E9CF0BB27869577956795B79508F478
:10697000B1609395C1F7BB0F58F711F460FFE8CFF2
:106980006F5F7F4F8F4F9F4FE3CF0C94CA3116F04C
:106990000C944B350C94853168940C947F310E9493
:1069A000AF31A8F39923C1F3AEF3DF93CF931F93D5
:1069B0000F93FF92C92FDD2788232AF02197660FB6
:1069C000771F881FDAF720E030E040E85FEB9FE3B5
:1069D000883920F0803E38F021968F770E9462320D
:1069E000E0E9F0E004C00E946232EDEBF0E00E94CA
:1069F0005E348B01BE01EC01FB2E6F57710975955A
:106A0000771F880B990B0E94B03028E132E741E3F1
:106A10005FE30E942231AF2D9801AE01FF900F91EC
:106A20001F91CF91DF910E9479320C949631FA0137
:106A3000DC01AA0FBB1F9B01AC01BF5728F4222722
:106A400033274427507820C0B75190F4AB2F00244F
:106A5000469537952795011CA395D2F3002071F038
:106A6000220F331F441FB395DAF30ED00C9461321A
:106A700061307105A0E88A07B94630F49B01AC018A
:106A80006627772788279078309621F020833183F6
:106A90004283538308959F3F31F0915020F48795AE
:106AA00077956795B795880F911D9695879597F976
:106AB0000895DB018F939F930E94E631BF91AF91C0
:106AC000A29F800D911DA39F900DB29F900D112448
:106AD0000895AA1BBB1B51E107C0AA1FBB1FA61725
:106AE000B70710F0A61BB70B881F991F5A95A9F777
:106AF00080959095BC01CD01089597FB072E16F463
:106B0000009407D077FD09D00E94693507FC05D0B5
:106B10003EF4909581959F4F0895709561957F4FB4
:106B20000895EE0FFF1F0590F491E02D0994DF9377
:106B3000CF931F930F939A9DF02D219FF00D8B9D66
:106B4000F00D8A9DE02DF10D039FF00D029FE00DE9
:106B5000F11D4E9DE00DF11D5E9DF00D4F9DF00D60
:106B60007F936F93BF92AF925F934F93D5010E9433
:106B700052328B01AC01D7010E945232EB01E80F77
:106B8000F91FD6010E94E6352F913F91D6010E9450
:106B90005232C60FD71FE81FF91FAF91BF910E9455
:106BA000E6352F913F910E945232C60FD71FE81F42
:106BB000F91FD6010E945232E60FF71F9801BE015D
:106BC000CF010F911F91CF91DF9108950E94523212
:106BD000460F571FC81FD91F08F4319608956894AF
:106BE00001C0E894F92FF12B12F00C942336A0E0A9
:106BF000B0E0EDEFF5E30C94FF31092E059422F49B
:106C00000E947F36112392F4F0E80F26FFEFE09404
:106C1000F09400951095B094C094D094A194BF0ABC
:106C2000CF0ADF0AEF0AFF0A0F0B1F0B0E942E3656
:106C300007FC0E947F36CDB7DEB7ECE00C941B3228
:106C4000689401C0E8948F929F92CF93DF930E9443
:106C50002E36DF91CF919F908F90089588249924AC
:106C6000F401E401B0E49F93AA279A158B049C04D5
:106C7000ED05FE05CF05D007A10798F4AD2FDC2F59
:106C8000CF2FFE2FE92D982C892E982F872F762F26
:106C9000652F542F432F322F2227B85031F7BF9141
:106CA00027C01B2EBF91BB27220F331F441F551F28
:106CB000661F771F881F991F881C991CEE1FFF1FD6
:106CC000CC1FDD1FAA1FBB1F8A149B04EC05FD050A
:106CD000CE05DF05A007B10748F08A189B08EC092C
:106CE000FD09CE09DF09A00BB10B21601A94E1F672
:106CF0002EF49401AF01BE01CD01000C0895609502
:106D000070958095909530954095509521953F4F81
:106D10004F4F5F4F6F4F7F4F8F4F9F4F0895002E04
:106D2000083090F0982F872F762F652F542F432F00
:106D3000322F22270850F4CF220F331F441F551F34
:106D4000661F771F881F991F0A95B2F7002D0895B7
:106D500097FD1094002E083098F00850232F342F00
:106D6000452F562F672F782F892F912DF4CF15940B
:106D70009795879577956795579547953795279573
:106D80000A95AAF71124002D08952A0D3B1D4C1DCC
:106D90005D1D6E1D7F1D801F911F08952A193B09DF
:106DA0004C095D096E097F09800B910B0895002441
:106DB000A7FD00942A1730054005500560057005B1
:106DC0008005900508950F931F93CF93DF93823032
:106DD000910510F482E090E0E0911706F09118061A
:106DE00030E020E0B0E0A0E0309799F421153105C3
:106DF00009F44AC0281B390B24303105D8F58A81A3
:106E00009B816115710589F1FB0193838283FE01EA
:106E100011C0408151810281138148175907E0F068
:106E20004817590799F4109761F012960C9312972E
:106E300013961C933296CF01DF91CF911F910F9142
:106E400008950093170610931806F4CF2115310505
:106E500051F04217530738F0A901DB019A01BD0137
:106E6000DF01F801C1CFEF01F9CF909318068093AD
:106E70001706CDCFFE01E20FF31F819391932250AD
:106E8000310939832883D7CF209115063091160612
:106E9000232B41F4209112013091130130931606F7
:106EA0002093150620911001309111012115310513
:106EB00041F42DB73EB74091140150911501241BA8
:106EC000350BE0911506F0911606E217F307A0F4D2
:106ED0002E1B3F0B2817390778F0AC014E5F5F4F30
:106EE0002417350748F04E0F5F1F50931606409346
:106EF0001506819391939FCFF0E0E0E09CCFCF9374
:106F0000DF930097E9F0FC01329713821282A0917F
:106F10001706B0911806ED0130E020E01097A1F4BB
:106F200020813181820F931F209115063091160622
:106F30002817390709F061C0F0931606E09315068B
:106F4000DF91CF910895EA01CE17DF07E8F54A8176
:106F50005B819E0141155105B1F7E901FB83EA838D
:106F600049915991C40FD51FEC17FD0761F4808139
:106F700091810296840F951FE9019983888382810C
:106F800093819B838A83F0E0E0E012968D919C913F
:106F900013970097B9F52D913C911197CD01029669
:106FA000820F931F20911506309116062817390776
:106FB00039F6309751F51092180610921706B093D3
:106FC0001606A0931506BCCFD383C283408151819E
:106FD000840F951FC817D90761F44E5F5F4F8881F2
:106FE0009981480F591F518340838A819B819383E4
:106FF00082832115310509F0B0CFF0931806E09394
:1070000017069ECFFD01DC01C0CF13821282D7CFBD
:10701000B0E0A0E0EEE0F8E30C94FB318C010097C7
:1070200051F4CB010E94E3368C01C801CDB7DEB725
:10703000E0E10C941732FC01E60FF71F9C0122508F
:107040003109E217F30708F49DC0D901CD91DC9115
:107050001197C617D70798F0C530D10530F3CE0188
:1070600004978617970708F3C61BD70B2297C1937F
:10707000D1936D937C93CF010E947F37D6CF5B0174
:10708000AC1ABD0A4C018C0E9D1EA0911706B09142
:107090001806512C412CF12CE12C109731F58091E0
:1070A0001506909116068815990509F05CC04616DC
:1070B000570608F058C08091100190911101009777
:1070C00041F48DB79EB74091140150911501841B76
:1070D000950BE817F90708F055C0F0931606E093F2
:1070E0001506F90171836083A0CF8D919C91119752
:1070F00012966C90129713967C901397A815B90569
:1071000059F56C0142E0C40ED11CCA14DB0420F115
:10711000AC014A195B09DA011296159780F0628278
:10712000738251834083D9016D937C93E114F10400
:1071300071F0D7011396FC93EE93129776CF2296B7
:107140008C0F9D1FF90191838083F301EFCFF093A2
:107150001806E093170669CF4816590608F42C0163
:107160007D01D3019ACFCB010E94E3367C010097C9
:1071700049F0AE01B8010E94CD38C8010E947F37A6
:10718000870153CF10E000E050CF91110895815650
:107190008A5108F4805285580895FB01DC0102C031
:1071A00001900D9241505040D8F70895FB01DC0149
:1071B00001900D920020E1F70895FB01DC014150A0
:1071C000504030F08D910190801919F40020B9F7EA
:1071D000881B990B0895FB01DC014150504048F099
:1071E00001900D920020C9F701C01D9241505040FE
:1071F000E0F70895FB0151915523A9F0BF01DC018F
:107200004D9145174111E1F759F4CD01019000204E
:1072100049F04D9140154111C9F3FB014111EFCFE8
:1072200081E090E00197089511E0C4E5D1E004C049
:10723000FE010E9491352196C535D107C9F7F89412
:10724000FFCF0000A040C80001011600640000004C
:10725000F0410000190680005E00BC007701FF01CC
:1072600086000000000079000000003B028201C897
:10727000018802F901D701EB0100000000450A185E
:107280000A740A4906110AFE09EF09000000004AC3
:10729000068201740A4906A606BE0631060D0A00DA
:1072A0002356657273696F6E3A00234C6F6767658A
:1072B00072204E616D653A0053484F57533D004769
:1072C000455400732000534156453D0054494D45F7
:1072D000493D0023496E74657276616C3D005449E6
:1072E0004D45443D00234475726174696F6E3D00E5
:1072F0004448543D0042543D00534C20503D005002
:107300006120756E6C696B656C7921006850610055
:107310004950414444002349503A004E45543D00F1
:1073200055565A002355562056303D005620004DE4
:10733000533D002C0023496E636F727265637421A4
:10734000204D533D31323344334435005428312CE1
:10735000322C33293D00206F43204453205468656C
:10736000726D6F6D657465720020572F6D5E32000F
:10737000555620496E74656E7369747900572F6D88
:107380005E32200055563D0070706D00434F323D17
:1073900000206E672F4C00504D28312E302C322E9D
:1073A000352C3130293D006F432000483D00250039
:1073B00068506120006F430020413D004C696768C0
:1073C0007420496E74656E7369747900206C78203E
:1073D000004C3D00495220466C616D65204C65763D
:1073E000656C3D00476173206C6576656C3D0020DF
:1073F0004D756C746973656E736F72730023456E9F
:1074000061626C65002344697361626C65002349A5
:107410006E76616C6964206B65792100424E4D4C3B
:107420003033004232683600234E6F2053656E734E
:107430006F72210057656C636F6D653A0023626D52
:1074400070206661696C65640073657269616C3A8D
:0C74500020002D35002D34002D330000ED
:107E0000112484B714BE81FFF0D085E080938100F7
:107E100082E08093C00088E18093C10086E0809377
:107E2000C20080E18093C4008EE0C9D0259A86E02C
:107E300020E33CEF91E0309385002093840096BBD3
:107E4000B09BFECF1D9AA8958150A9F7CC24DD24C4
:107E500088248394B5E0AB2EA1E19A2EF3E0BF2EE7
:107E6000A2D0813461F49FD0082FAFD0023811F036
:107E7000013811F484E001C083E08DD089C08234E0
:107E800011F484E103C0853419F485E0A6D080C0E4
:107E9000853579F488D0E82EFF2485D0082F10E0AE
:107EA000102F00270E291F29000F111F8ED06801E7
:107EB0006FC0863521F484E090D080E0DECF843638
:107EC00009F040C070D06FD0082F6DD080E0C81688
:107ED00080E7D80618F4F601B7BEE895C0E0D1E017
:107EE00062D089930C17E1F7F0E0CF16F0E7DF06D8
:107EF00018F0F601B7BEE89568D007B600FCFDCFD4
:107F0000A601A0E0B1E02C9130E011968C91119780
:107F100090E0982F8827822B932B1296FA010C0160
:107F200087BEE89511244E5F5F4FF1E0A038BF0790
:107F300051F7F601A7BEE89507B600FCFDCF97BE46
:107F4000E89526C08437B1F42ED02DD0F82E2BD052
:107F50003CD0F601EF2C8F010F5F1F4F84911BD097
:107F6000EA94F801C1F70894C11CD11CFA94CF0C13
:107F7000D11C0EC0853739F428D08EE10CD085E9AC
:107F80000AD08FE07ACF813511F488E018D01DD067
:107F900080E101D065CF982F8091C00085FFFCCF94
:107FA0009093C60008958091C00087FFFCCF809118
:107FB000C00084FD01C0A8958091C6000895E0E648
:107FC000F0E098E1908380830895EDDF803219F02E
:107FD00088E0F5DFFFCF84E1DECF1F93182FE3DFCA
:107FE0001150E9F7F2DF1F91089580E0E8DFEE27F6
:047FF000FF270994CA
:027FFE00040479
:00000001FF
